:020000040800F2
:1000000068200020B501000801020008A9180008B6
:1000100001020008010200080102000800000000BF
:1000200000000000000000000000000001020008C5
:10003000010200080000000001020008010200089F
:100040000102000801020008010200080102000884
:100050000102000801020008010200080102000874
:100060000102000801020008010200080102000864
:100070000102000801020008010200080102000854
:100080000102000801020008010200080102000844
:100090000102000801020008010200080102000834
:1000A0000102000801020008010200080102000824
:1000B000010200080102000801020008C51300083F
:1000C000D1130008DD130008E9130008010200083D
:1000D00001020008010200080102000801020008F4
:1000E00001020008010200080102000801020008E4
:1000F00001020008010200080102000801020008D4
:1001000001020008010200080102000801020008C3
:1001100001020008010200080102000801020008B3
:1001200001020008010200080102000801020008A3
:100130000102000801020008010200080102000893
:100140000102000801020008010200080102000883
:100150000102000801020008010200080102000873
:100160000102000801020008010200080102000863
:100170000102000801020008010200080102000853
:040180000102000870
:1001840041A3525576332E302D6265746131312D81
:1001940038342D673532376464626500000000002E
:0F01A4000000000035323764646265000000011E
:1001B400002100F004B80C4B5B58435004310B4849
:1001C4000B4B42189A42FFF4F6AF0A4A00F003B808
:1001D400002342F8043B084B9A42FFF4F9AF01F0C4
:1001E4009DFE01F091FB70478CAB000800000020DD
:1001F400140000201400002068000020FFF7FEBF58
:1002040030B501208BB002F0E5FA002401902546B8
:10021400E0B200F0BBFB01AB08B9185519E01A5D58
:10022400042A10DD164800F025FD02A920220198B9
:1002340001F03CFE02A800F01DFD0120002102F0A7
:10024400B9FA00201AE00132D2B2052A1A55A8BF21
:1002540001250134042CDBD1019C54B1094800F080
:1002640009FD204602A9202201F020FE02A800F088
:1002740001FD0120214602F09DFA28460BB030BD55
:1002840048A4000874A4000808B500F087FA80F0B8
:100294000100C0B208BD000008B54FF480610348F6
:1002A40002F073F8003018BF012008BD00180240A6
:1002B4002DE9F0434A4D89B0284600F00BFD28464D
:1002C4000D21052208AE02F06BF8052228460E2106
:1002D40002F066F84FF4005346F81C3D0024012751
:1002E4004FF00209284631468DF80A408DF80B403C
:1002F4008DF808908DF8097001F0FEFF4FF48043EB
:1003040028463146019301F0F7FF4FF48053284605
:10031400314601934FF400788DF808408DF80A4077
:1003240001F0EAFF284631468DF808408DF80B703D
:10033400CDF8048001F0E0FF4FF480632846314695
:1003440001938DF808408DF80B4001F0D5FF4FF470
:1003540080732846314601938DF808708DF80B4060
:1003640001F0CAFF4FF40043284631460193A5F536
:1003740044451C4E8DF80A708DF80B4001F0BCFF0B
:1003840039464FF4001002F0B9F9174B3360284690
:1003940002F030FA03A802F0A4FA4FF44043ADF897
:1003A4000C3039464FF482733068ADF80E30ADF836
:1003B4001040ADF81290ADF81470ADF8168001F04D
:1003C40019F803A9ADF818002846ADF81A4002F050
:1003D40069FA2846394602F090FA09B0BDE8F0837C
:1003E40000180240140000200024F40008B5022084
:1003F40001F046FD012000F0B7FA022001F040FDB3
:100404000120BDE8084000F09DBA000010B5044684
:100414000548022102F07FFA0028F9D0214602485B
:10042400BDE8104002F075BA0054014038B501220D
:1004340004460D4628484FF4807101F0ACFF0120BA
:1004440001F01EFD24484FF40041002201F0A3FFF7
:100454004FF480710022204801F09DFF012001F03B
:100464000FFD4FF400411C48012201F094FF0120CC
:1004740001F006FD18484FF4007101F086FF18B131
:100484001648174A68210AE013484FF4004101F066
:100494007CFF08B1254404E01048124A692101F0A8
:1004A400A9FCAC4204D014F8010BFFF7AFFFF8E746
:1004B40009484FF48071012201F06DFF08240020E7
:1004C400FFF7A4FF013CFAD103484FF40071BDE8E3
:1004D400384001F05ABF00BF001802408DA4000844
:1004E40097A40008B2A4000810B54FF48071044624
:1004F4000022054801F04FFF642001F0BBFC2046B8
:10050400BDE81040FFF782BF0018024008B5074855
:10051400802102F000FA0028F9D105484FF48071D7
:100524000122BDE8084001F036BF00BF005401407D
:100534000018024010B540F2F514FFF7ADFE50B1BB
:10054400013C04D1054800F095FB204610BD642011
:1005540001F090FCF1E7012010BD00BFCFA400081A
:1005640010B504460420FFF7BFFF2046FFF74EFFF7
:10057400BDE81040FFF7CABF10B504460120FFF7DD
:10058400B3FFE0B2FFF742FFC4F30720FFF73EFFDB
:10059400C4F30740FFF73AFF200EFFF737FFBDE82B
:1005A4001040FFF7B3BF000010B5FFF781FE1848F5
:1005B40047F6DE01FFF73AFFFFF718FF002401209A
:1005C400FFF7CEFFFFF7B6FF78B10320FFF78CFFEC
:1005D400FFF79CFF0F4800F063FB204600F06EFB22
:1005E4000D48BDE8104000F045BB094847F6DE0160
:1005F4000134FFF71BFF152CE1D1084800F03AFB4A
:100604000220FFF771FFBDE81040FFF77FBF00BF76
:10061400262A0008F2A400080DA5000817A5000862
:1006240008B55D224B1C504300EB5300074BB0FB55
:10063400F1F01A78C0B2824207D01870FFF79CFF1D
:100644000220BDE80840FFF78BBF08BD0000002072
:1006540008B5FFF791FF0320BDE80840FFF780BF0E
:1006640008B50220FFF740FFBDE80840FFF74EBF82
:1006740001F1C04102F0C4B970B543489AB000F02A
:1006840029FB424800F026FB414800F023FB414B84
:1006940093E8030001AC84E803003C48214601F0E0
:1006A4002BFE3A480421012201F075FE00250223A5
:1006B400029535488DF80830072103230C228DF864
:1006C4000930019501F06CFE80232F4801932146E7
:1006D40001F012FEEBB2022B04D02C48A9B20C227A
:1006E40001F05EFE0135102DF4D14FF6FB7327485F
:1006F4000193214601F000FE0226314601362448CA
:100704000C22B6B201F04CFE102EF6D14FF6FC735B
:1007140021461F48019301F0EFFD042100221B48EC
:100724001D4D01F038FE0A2001F0A4FB0122042132
:10073400164801F030FE1E2001F09CFB012001460A
:1007440001F0C4FF0FCD03AC0FC495E8070084E8A3
:100754000700402200210AA802F05BF902230B9350
:1007640008230C934FF4805312934FF400531393C4
:100774000AA803AB18930D9601F03CFD002001215B
:1007840001F0AAFD1AB070BD00040240000C024042
:100794000010024004A300080CA300080E4B98228A
:1007A4001A80A3F68A231B88DBB2512B07D10B4B8B
:1007B4001888C0B2B0F152025042504100E000200B
:1007C40030B1074B1888C0B2B0F1590358425841B0
:1007D400014BF0221A807047AA0A006022000060D0
:1007E4002400006002460B460420502100F0C9BDDD
:1007F40002460B460420502100F0D8BD032873B5EF
:100804000E4603D0042804D001F00AFB14251C4C26
:1008140001E01C4C162528460DF10701FFF7E2FF05
:1008240008B900202AE02378AEB10BB1013323E0EC
:100834009DF8071021F0060141F0020128468DF8C9
:100844000710FFF7D5FF0028EBD001250320257002
:1008540001F016FB11E05AB2012A0CDC9DF80710D6
:10086400284601F0F9018DF80710FFF7C1FF0028B1
:10087400D7D0267001E0013B2370012002B070BD87
:10088400180000201900002073B5254800F022FA52
:1008940002254FF410730024012621480093694671
:1008A4008DF804508DF805508DF806608DF80740DA
:1008B40001F022FD1A480621042201F071FD0422F0
:1008C4000921174801F06CFD154800F01DFA154880
:1008D40000F000FA42F20C036946124800938DF8C6
:1008E40005508DF804608DF806408DF8074001F03E
:1008F40003FD0C4800F008FA042000F0DFFC204659
:100904006946FFF76FFF9DF80050B54205D10320FB
:100914002946FFF773FF284600E0204602B070BD69
:10092400000402400014024010B50446042000F004
:10093400C5FC21460420FFF761FF0420BDE81040F8
:1009440000F0EABC38B5074C0546204600F0C2F971
:1009540020462A46042101F01EFD2046BDE8384009
:1009640000F0D2B90014024038B5074C05462046C1
:1009740000F0B0F920462A46082101F00CFD20467B
:10098400BDE8384000F0C0B90014024038B5094C45
:1009940004EB0014606800F09DF92189606801F09F
:1009A400F4FC0546606800F0AFF9D5F1010038BFEA
:1009B400002038BD28A3000838B500242546E0B23D
:1009C400FFF7E4FFA04001340543042CEDB2F6D157
:1009D400284638BD73B54FF480400121154C01F011
:1009E4008DFE04F1400654F80A0C00F073F96846D1
:1009F40001F0C2FC02238DF80530237854F80A0C68
:100A04008DF80730694654F8063C009300258DF8AC
:100A14000450103401F070FC54F81A0C00F074F90E
:100A2400B442E0D14FF48040294601F067FE02B0A1
:100A340070BD00BF36A3000808B5054B1B781BB971
:100A44000448322101F0E2F9BDE8084001F012BB8C
:100A54001A0000204AA50008114B1B7870B5054602
:100A64000C461BB90F48382101F0D0F9032906D9E7
:100A74008E083146FFF7E0FFB6003544A41B1CB9CD
:100A8400BDE8704001F004BB00231846EA5C013362
:100A9400A34242EA0020F9D1BDE8704001F0E4BA73
:100AA4001A0000204AA50008024B1A780AB901224C
:100AB4001A7070471A00002008B5084B1A781AB942
:100AC40007482B2101F0A2F901214FF480505970FD
:100AD40001F0F0FDBDE8084001F0C0BA1A000020A2
:100AE4004AA5000808B5074B1A781AB906485121D7
:100AF40001F08CF9002159704FF48050BDE8084092
:100B040001F0D8BD1A0000204AA5000870B50C46B3
:100B14000546A608FFF7D0FF28463146FFF78CFFAD
:100B240004F0030105EB8600FFF796FF0446FFF788
:100B3400D9FF204670BD70B5A0B00D460646FFF73C
:100B4400BBFF2C467119802CC4EB0101684608D9FF
:100B54008022FFF78DFD68462021FFF76DFF803C62
:100B6400F0E72246FFF784FD21466846FFF774FF4D
:100B74000446FFF7B7FF204620B070BD2DE9F041D1
:100B8400284C86B0204600F0A5F84FF480200121BF
:100B940001F0A8FD20460A21072201F001FC06AE5F
:100BA400072220460B2101F0FBFB002501274FF013
:100BB40002084FF48063204669468DF8065046F8D3
:100BC400183D8DF807708DF804808DF8058001F0CC
:100BD40093FB4FF400632046694600938DF804802C
:100BE40001F08AFBADF80C50ADF80E50ADF8105082
:100BF400ADF814500C4D4FF46133029328460C2386
:100C040002A9ADF8123001F08DFE2846394601F0F4
:100C1400E1FE204600F078F8044B1F7006B0BDE8F2
:100C2400F08100BF00080240004800401C00002082
:100C3400084B1B7810B504465BB10748402101F00E
:100C4400D9FE0028F9D021460348BDE8104001F040
:100C5400CDBE10BD1C0000200048004008B5FFF7C1
:100C6400E7FF0348402101F0C5FE0028F9D008BD84
:100C740000480040094B1B7810B573B1441E14F8AA
:100C8400010F10B1FFF7EAFFF9E70D20FFF7E6FFC8
:100C94000A20BDE81040FFF7E1BF10BD1C00002092
:100CA400054B1B7810B533B1441E14F8010F10B175
:100CB400FFF7D4FFF9E710BD1C0000201FB50C227C
:100CC40001A901F0F3F801A8FFF7EAFF05B05DF808
:100CD40004FB000000F13F4000F57E00C0F38720D4
:100CE40008280BD8064A135C591C115433B9054B18
:100CF40001211A6B01FA00F010431863704700BF1A
:100D04001D0000200038024000F13F4000F57E0045
:100D1400C0F3872008280ED8074A135C5BB1013B57
:100D2400DBB213543BB9054B01211A6B01FA00F0F5
:100D340022EA0000186370471D00002000380240BA
:100D440002460068838823F4E0631B041B0C838041
:100D540003889BB243F40073038008230020517579
:100D640013751076704737B504460D46FFF7B2FF8A
:100D74000023204669468DF804308DF805308DF83F
:100D84000730009501F0B8FA2046FFF7BDFF03B025
:100D940030BD00000A4B10B5342400FB0434236B2F
:100DA4006BB10A2001F06CF86068A168FFF7DBFF03
:100DB40020696169FFF7D7FF236B0120984710BDB5
:100DC40070A30008F7B5044616460D461F46FFF704
:100DD40081FF022001238DF804008DF805008DF8B1
:100DE40006302046002369468DF80730009501F04F
:100DF40083FA204631463A4601F0D2FA2046FFF7FC
:100E040083FF03B0F0BD0000037D082B10B504463A
:100E140007D10268938823F4C0631B041B0C9380DE
:100E240083E0434A006802EB8303996E01F08CFB74
:100E340000287AD0237D072B71D8DFE803F0040B58
:100E44001A22323A596D227A236802F0FE021A827B
:100E5400012305E02368A27A1A82627A12B102237E
:100E6400237562E09A8892B242F480629A800623E3
:100E7400F6E723681A8892B242F480721A80032338
:100E8400EEE7237A226843F001031382E37A012B0D
:100E940005D1138823F480631B041B0C13800423E3
:100EA400DEE723689A8892B242F480629A8005232E
:100EB400D6E72368227B198A23699954237BE27A33
:100EC4000133DBB2591C9142237307D12268138882
:100ED40023F480631B041B0C138026E0934224D16B
:100EE4002268938823F480631B041B0C938013E013
:100EF400217B236922685B5C1382237BE17A0133C3
:100F0400DBB29942237310D1938823F480631B04CA
:100F14001B0C93800723A3E72046012101E0204610
:100F24000021BDE81040FFF70BBF002010BD00BF3B
:100F340070A300087FB51D4E1C2303FB0063054608
:100F44001B790BB9FFF726FF194B342405FB043436
:100F54006068A168A289A37BFFF734FF228BA37E7C
:100F640020696169FFF72EFFE069012101F0BAFBF6
:100F7400684601F0C3FA0F4A236A009393424FF480
:100F84008063ADF80A304FF01C0303FB05F588BFFE
:100F9400626A705988BFADF80620694601F040FACC
:100FA4007059012101F0B8FA04B070BD2800002086
:100FB40070A30008A086010073B504460E46002500
:100FC400FFF788FE0123204669468DF80430009619
:100FD4008DF805508DF8075001F08EF92046B1B216
:100FE4002A4601F0D8F92046FFF78EFE02B070BD04
:100FF400094B10B5342400FB0434236B5BB100208F
:1010040098476068A168FFF7D7FF20696169BDE868
:101014001040FFF7D1BF10BD70A300081C23104A75
:10102400434370B50546D058D61801F0CBF90D4BA3
:10103400342405FB04340021E06901F053FB3379C7
:1010440023B92846BDE87040FFF7D2BF6068A168A5
:10105400FFF789FE20696169BDE87040FFF783BE30
:101064002800002070A300082DE9F74F4A4E9B4644
:1010740096F838300F469246B0461BB9474840F2BE
:10108400951104E0042804D944484FF4CB7100F0CE
:10109400BDFE434B18444FF01C0990F8885009FBDF
:1010A40005F906EB090423790BB9002071E056F821
:1010B4000900038B980713D49DF830306772E372EC
:1010C40000270D9B84F808A084F80AB027732775BD
:1010D4002361E78256F80900012101F029FA20E092
:1010E4002846FFF79BFF2846FFF724FF56F8092000
:1010F4002C48138B9907DFD50138FAD1D5E7227E26
:1011040022B1019A511E0191002AF8D100222276BF
:10111400019A02B3227D082A13D1677D237D082B0F
:1011240026D023681A8892B242F480721A809A8870
:1011340092B242F440729A8001222276194A0192B4
:10114400DFE7E28AB2F57A7F05D20132E28201203A
:1011540000F096FEE2E79A8822F4E0621204120C90
:101164009A801A8892B242F400721A800823237576
:101174001C236B4358F803100A4B0A8B920707D5BC
:10118400013BFAD12846FFF749FF2846FFF7D2FE74
:10119400384603B0BDE8F08F2800002050A50008B1
:1011A40070A3000880841E00017D0368082906D10D
:1011B4009A8822F480721204120C9A8036E09A8A79
:1011C400120505D59A8A22F400621204120C9A823E
:1011D4009A8AD20505D59A8A22F480721204120CD6
:1011E4009A829A8A52051ED59A8A22F4806212043F
:1011F400120C04299A820AD1032202759A8822F4D5
:10120400E0621204120C9A80002303760EE0012996
:1012140009D19A8822F4E06212040021120C0175AB
:101224009A80017602E00021FFF78ABD0020704712
:101234002DE9F3411E4D1F4C0026DFF87C802B68FE
:1012440044F80C3C1C2202FB0682002304F8083CF0
:1012540013760822227295F828208DF8042001279D
:101264000C2201A8237004F8013C63608DF805206A
:101274008DF806308DF8077000F0BAFE95F8293025
:101284008DF8043001A800F0B3FE3E4454F80C0C71
:1012940001F098F8022E05F1340504F11C04CCD1B8
:1012A400384688F83870FFF7A3FE02B0BDE8F08135
:1012B40070A300083400002028000020124A13B54F
:1012C40092F83810034621B9104840F2331100F067
:1012D4009DFD042807D9052200920C480C4A40F2CF
:1012E400351100F087FD0B490B441C2493F888004A
:1012F40004FB002423790BB9FFF71CFE2379013387
:10130400237102B010BD00BF2800002050A50008C2
:1013140056A5000870A3000808B5104B93F83820B0
:101324001AB90F4840F2451104E0042804D90C48C6
:101334004FF4A37100F06AFD0A4A10441C2290F88D
:10134400880002FB003213793BB1013BDBB213711D
:101354001BB9BDE80840FFF761BE08BD28000020A6
:1013640050A5000870A3000873B5069C00930E46B0
:1013740015460194012132462B46FFF775FE02B053
:1013840070BD07B500930123FFF7EEFF03B05DF8CE
:1013940004FB73B5069C00930E4615460194002188
:1013A40032462B46FFF760FE02B070BD1FB504AC99
:1013B40004F8013D01230094FFF7EBFF04B010BDD6
:1013C4000148FFF721BD00BF280000200148FFF7B6
:1013D400EBBE00BF280000200148FFF715BD00BF89
:1013E400440000200148FFF7DFBE00BF4400002096
:1013F400FFF79ABA30B585B004460D46684601F049
:1014040015F90DB9029805E0012D01D1039801E009
:1014140000F006FDB4EB500F0ED8B0FBF4F000F072
:1014240039FD002802DC0748272103E0082804DDF1
:101434000448282100F0EAFC01200138C00080B2F1
:1014440005B030BD82A50008B0F1006F10B50446A8
:101454000BD20D48FFF724FC2046FFF72FFC0B4866
:10146400FFF71EFC4FF0FF3010BD094A002352F86D
:10147400041FA14202D851688C4202D301330B2BC2
:10148400F5D1184610BD00BFFAA5000888A50008CC
:10149400FCA300082DE9F04705462D480F461646E3
:1014A4009946FFF7FDFB2846FFF708FC2948FFF79C
:1014B400F7FB3846FFF702FC2748FFF7F1FB002F44
:1014C4003FD02846FFF7C0FF0446781E2844FFF7A4
:1014D400BBFF002C074637DB002835DBC4EB0008D4
:1014E40008F101081EB1002041464A46B04700F009
:1014F400E1FD1A4B012503EB440ABC421FDCF32037
:1015040000F0EEFD0AEB4503002133F8020C00F075
:101514001FFE09280BD01248FFF7C2FB2046FFF735
:10152400CDFB1048FFF7A6FB00F0D2FD0CE01EB186
:10153400284641464A46B04701340135DDE700F00C
:10154400C7FD0120BDE8F0870020BDE8F08700BF9B
:10155400A3A50008B7A50008BAA5000830A4000890
:10156400BEA50008EDAA00082DE9F84606461F4866
:1015740015468A461F46FFF793FB3046FFF79EFB4E
:101584001B48FFF78DFB2846FFF798FB1948FFF728
:1015940087FB00F08FFDF32000F0A2FD4FEAD51980
:1015A4000024AC421DD0A0191AF8041000F006FE65
:1015B40009280DD01048FFF773FB3046FFF77EFB78
:1015C4000E48FFF757FB00F083FD0020BDE8F886C6
:1015D4002FB1630603D1E0094946089AB84701349C
:1015E400DFE700F075FD0120BDE8F886D6A5000808
:1015F400B7A50008BAA50008EAA50008EDAA0008E6
:1016040008B545F2555000F0ABFF042000F0AEFFE2
:1016140040F6FF7000F0B0FF002000F0A1FF4FF48F
:1016240080500121BDE8084000F038BD08B500F045
:10163400B1FFBDE8084000F0A5BF08B57D2001F06A
:10164400A5F8003018BF012008BD4900FEF7E8BF27
:101654004B0803EB5000FEF7E3BF000070B586B003
:101664000446FFF721FA01210020FEF7D9FF0420E8
:1016740000F020FB03A8214600F06EFB03A800F055
:101684007AFB08B928480BE02848FFF7F3FA04F17D
:101694000C000499FFF74FFA059B984204D02448A4
:1016A400FFF7E8FA01203DE0049D2248FFF7E2FA43
:1016B4002946214A21480023FFF7ECFE049E2048D6
:1016C400FFF7D8FA002504F1C0411E4B00953246BD
:1016D4000C311A48FFF748FF1B48FFF7E1FA04985A
:1016E400FFF7ECFA1948FFF7DBFA04991348FFF700
:1016F4000DFA04461648FFF7D3FA0598FFF7DEFA09
:101704001448FFF7CDFA2046FFF7D8FA1248FFF73E
:10171400B1FA059B9C4204D01048FFF7ABFA0220B3
:1017240000E0284606B070BD03A6000821A6000804
:101734003EA6000861A600084F1600080000010834
:1017440074A600085516000887A6000895A6000888
:101754009EA60008B1A60008EDAA0008B7A60008D6
:1017640008B5022000F0BEFAD8B3042000F0BAFA9B
:1017740070B11C48FFF77EFA042000F0A7FA02209B
:1017840000F0A4FA4FF40040BDE8084000F09EBA0F
:101794001548FFF76FFA082000F098FA102000F0BF
:1017A40095FA202000F092FA402000F08FFA4FF4CE
:1017B4008010FFF753FF022807D1082000F07AFABF
:1017C400102000F077FA00F04DFB042000F07EFAC0
:1017D400022000F07BFA4FF40040BDE8084000F01E
:1017E40069BA08BD02A7000838A7000810B5254843
:1017F400FFF740FA4FF40010FFF730FF10B1022852
:101804003AD809E0202000F061FA402000F05EFAA6
:10181400802000F04FFA2FE0082000F04BFA10204F
:1018240000F048FA202000F05DFA20B91648FFF7CE
:1018340021FA202007E0402000F054FA58B9134858
:10184400FFF718FA402000F035FA4FF4007000F06A
:1018540031FA00F007FB0E48FFF70CFA082000F0FD
:1018640035FA102000F032FA202000F02FFA402040
:1018740000F02CFA002400E00124042000F026FAF1
:10188400204610BD53A700086DA70008A6A70008AE
:10189400DFA7000808B50248FFF7ECF900F0E7FA03
:1018A40019A800081EF0040F0CBFEFF30880EFF333
:1018B4000980FFF7EFBF70471FB504461048FFF7D4
:1018C400D9F901A90C22204600F0F0FA01A8FFF78B
:1018D400D1F92046FEF7BCFEFFF76EF8094B20F065
:1018E400040018701C46FFF767F8237800F0FB002B
:1018F400834201D000F0B6FA0A2000F0C1FAF2E700
:101904000FA80008640000207FB54FF0805001212B
:1019140000F0E8FE022000F04BFE012807D102206F
:1019240000F050FE9248FFF7A5F900F0A0FA00215C
:101934004FF0805000F0D6FEFFF720F98D48FFF7F6
:1019440099F98D48FFF796F98C48FFF793F98C487D
:10195400FFF790F98B48FFF78DF98B48FFF78AF969
:101964008A48FFF787F98A48FFF784F98948FFF71F
:1019740081F98948FFF77EF9FFF75AFCFEF784FFE7
:1019840000F0BAF900F0D0F900210C2201A801F00E
:1019940040F800F0C5F901A90C2200F087FA01A86B
:1019A400FFF768F97348FFF765F97248FFF762F9C2
:1019B4004FF4804000F096F990B17848FFF75AF957
:1019C4004FF4804000F082F9082000F07FF91020E5
:1019D40000F07CF9202000F079F9402000F076F93D
:1019E400FEF74AFEFEF7F6FFFEF7DEFDFEF708FC03
:1019F40008B16B4803E0FEF747FC10B16948FFF7F4
:101A04005BFF00F08CF9802000F06CF918B18020A5
:101A140000F05CF954E04FF4003000F063F9044640
:101A240020B14FF4003000F051F92EE10120FEF70F
:101A3400ADFFB0B12046FEF7A9FF90B15A48FFF7B9
:101A440019F941F288340120FEF7A0FF98B1002073
:101A5400FEF79CFF78B1012000F012FA013CF2D1AC
:101A640013E1524B0CCB013301D0013203D1504866
:101A7400FFF700F909E1FFF7E0FD18B3FFF7DDFD1B
:101A840010B14C48FFF7F6F84FF4007000F02AF953
:101A940010B14948FFF7EEF84FF4007000F016F962
:101AA400102000F01FF9D0B14448FFF7E3F80820F4
:101AB40000F00CF9102000F009F9FFF797FEF8B9CF
:101AC4003F489CE74FF4007000F00CF90028D5D192
:101AD400082000F0FBF8102000F0F8F80EE00820D1
:101AE40000F000F920B13748FFF7C4F8102003E0F4
:101AF4003548FFF7BFF8082000F0DCF8FFF730FEA8
:101B04004FF4005000F0EEF804464FF4805000F01B
:101B1400E9F8400040EA84044FF4006000F0E2F881
:101B2400E4B22043C3B2072B0DD14FF4006000F0A0
:101B3400CDF84FF4805000F0C9F84FF4005000F095
:101B4400C5F822485BE70133DBB2023B4FF4006087
:101B5400052B41D8DFE803F03C4003403C4000F053
:101B6400B5F84FF4805000F0B1F84FF4005033E072
:101B740024A80008EDAA000831A8000848A8000815
:101B840061A800088FA80008BEA80008EEA80008F5
:101B94001FA9000851A9000883A90008B4A90008D6
:101BA400014550FE024550FEE1A90008000001086D
:101BB40013AA000826AA00083EAA00085EAA000884
:101BC400034550FE86AA0008ACAA0008044550FE4E
:101BD40000F07CF84FF4805000F06CF8FFF710FD33
:101BE400FFF724FD2B4B2C485D681E68FFF758F85F
:101BF4002846FFF763F82948FFF752F800239A00B4
:101C040002F1604202F5614201334FF0FF31082BCB
:101C1400C2F88010C2F88011F1D1214B4FF4801228
:101C240000241A635C639C631C645C6400F0DAFC4B
:101C34001C48012100F06EFD21461A4800F06AFD9F
:101C4400F120012100F072FD2146F12000F06EFD2B
:101C54000120014600F076FD2146012000F072FDCE
:101C64001148012100F07AFD21460F4800F076FD6D
:101C74000E48012100F07EFD0C48214600F07AFD5B
:101C840063B64FF0FF3EB54628470948FEF7F2FF1A
:101C940013E700BF00000108D2AA0008E6AA000862
:101CA400003802400010E022FFC9FEF6337F7704BB
:101CB400EEAA000810B50446002000F08BFD40EAAF
:101CC40004010020BDE8104000F074BD10B50446C6
:101CD400002000F07FFD20EA04010020BDE8104050
:101CE40000F068BD10B50446002000F073FD2042EA
:101CF4000CBF0020012010BD08B54FF08050012119
:101D040000F0F0FC012000F04DFC0120FFF7EAFF99
:101D140020B90121BDE8084000F04CBD08BD704762
:101D2400022000F057BD000008B5FFF7F9FF054B8E
:101D34001968884204D00220BDE8084000F03ABD8A
:101D440008BD00BF8401000808B50248FEF792FFF1
:101D540000F088F80DAB00081FB504460C2201A85A
:101D6400FEF786FC01AB03CB20601868A060204618
:101D7400616004B010BD0068B0F10C0358425841D2
:101D84007047000080B50546174610480E461C46AD
:101D9400FEF786FF3846FEF783FF0D48FEF780FF07
:101DA4002846FEF77DFF0B48FEF77AFF3046FEF724
:101DB40085FF2CB10848FEF773FF2046FEF770FF3D
:101DC4000648FEF757FFFFF7BFFF00BF2AAB000826
:101DD40033AB000836AB000834AB0008EDAA0008AA
:101DE4001FB506AA52F8044B039200921A462346E2
:101DF400FFF7C8FF0CB41FB506AA52F8043B0392C0
:101E04000092014AFFF7BEFF38AB000807B5002374
:101E140000937246014BFFF7E3FF00BF3FAB00089E
:101E2400744608B50548FEF73BFF2046FEF746FF1B
:101E34000348FEF71FFFFFF787FF00BF47AB00080B
:101E4400EDAA0008BFF34F8F044A054BD16801F493
:101E5400E0610B43D360BFF34F8FFEE700ED00E07A
:101E64000400FA0508B5FEF7FBFBFFF7EBFF08B526
:101E7400FFF7E8FF1623584301387FF4FDAF70479E
:101E840010B504462CB14FF47A70FFF7F3FF013C10
:101E9400F8E710BD10B5B0FA80F400F029F8012875
:101EA4000CBFC4F11F00C4F1200010BD0A2A30B5D4
:101EB4001DDD0C46302304F8023B78234B700023CD
:101EC4009D00C5F11C050F22AA400240EA40092AE0
:101ED40001D8303202E00F2A02D85732D2B200E0E1
:101EE4002022E2540133082BEAD100238B7230BD47
:101EF40000F0AA33A0EB530000F0CC3300F03330F1
:101F040000EB930000EB101000F00F3000EB1020FA
:101F140000EB104000F03F00704700002D4BD3F859
:101F2400882042F47002C3F888202B4B1A680021E1
:101F340042F001021A6099601A6822F0847222F455
:101F440080321A60254A5A601A6822F480221A6084
:101F5400D9601A6C42F080521A64214A116841F423
:101F6400404111609A689A609A689A609A6842F44B
:101F740080529A601B4A5A601A6842F080721A6052
:101F84001968154A8901FBD5174B40F203611960A2
:101F9400936823F003039360936843F00203936010
:101FA4000D4B9A6802F00C02082AF9D19A6822F4BF
:101FB40000029A600D4AC3F884201A6842F08062D5
:101FC4001A60054B1B681B01FBD5024B4FF00062E6
:101FD4009A60704700ED00E00038024010300024A1
:101FE400007000401040010F003C024000300050DF
:101FF400C278037810B50AB3164A4478D268D2433B
:10200400C2F30222C2F10401C9B204FA01F10F249D
:1020140044FA02F28478C9B222400A4303F16043CD
:1020240003F561431201D2B283F80023037801223D
:10203400590903F01F0302FA03F306E059090122C8
:1020440003F01F0302FA03F32031034A42F821305C
:1020540010BD00BF00ED00E000E100E0014B0122F3
:102064009A60704700300240014B1860186870474E
:102074000030024000EB81018842044B03D050F849
:10208400042B1A60F8E71868704700BF003002405C
:10209400014B1868704700BF00300240044B9A6837
:1020A40009B1104301E022EA00009860704700BFC4
:1020B400002004E0044B1A69002A04DA034A5A6037
:1020C40002F188325A607047003C024023016745A0
:1020D400024B1A6942F000421A617047003C024008
:1020E400014BD860704700BF003C02400E4BDA68D9
:1020F400D00310D4DA68D1060FD4DA68D2050ED42E
:10210400DA6812F0EF0F0CD1DB6813F0020F0CBF8A
:1021140009200820704701207047062070470220DC
:1021240070470720704700BF003C024007B50923F1
:102134008DF80730FFF7DAFF8DF807009DF80730B8
:10214400012BF7D09DF8070003B05DF804FB0000F5
:1021540070B5064641B1012908D0022914BF4FF4D5
:1021640040754FF4007503E00D4601E04FF48075AF
:10217400FFF7DCFF09281ED10F4C236923F44073B9
:10218400236121690D432561236923F0F803236149
:10219400236943F002031E432661236943F4803319
:1021A4002361FFF7C3FF236923F00203236123693B
:1021B40023F0F803236170BD003C024070B505466E
:1021C4000E46FFF7B3FF092811D1094C236923F404
:1021D4004073236123692361236943F0010323616D
:1021E4002E70FFF7A3FF236923F00103236170BD61
:1021F400003C024070B543688568846A0168426B9C
:1022040045EA0306C3681E4303691E4343691E432C
:1022140083691E43C3691E43036A1E43436A3343EF
:1022240043EA0406C36A1E43036B334343EA0206CC
:102234008B0003F12043082D1E6003D11D6845F077
:1022440040051D60B2F5801F836B12D189B14FF038
:1022540020425668156845F480151560156845F4E4
:10226400807515601D6926F47006013D46EA055522
:1022740055601A689D6915435A6845EA02159A68BB
:1022840045EA0225DA6845EA02451A695B6945EAC6
:10229400025242EA03624E1C4FF02043B4F5804FD1
:1022A40043F8262010D1C36B1A68986910435A6802
:1022B40040EA02109A6840EA02201A695B6940EA1F
:1022C400025242EA036201E06FF07042014B43F8AC
:1022D400212070BD040100A0800000F1204019B14C
:1022E400036843F0010302E00268024B13400360F9
:1022F400704700BFFEFF0F002DE9F0410F68002377
:1023040001229A4002EA0705954230D15A0003247B
:1023140006689440E443264006600E79D0F800C075
:1023240006FA02F8013E48EA0C0C012EC0F800C07F
:1023340014D8866891F805C02640866086680CFA31
:1023440002FC4CEA06068660466826EA05054560F6
:102354008D7946689D40ADB235434560C5682C40D3
:10236400C460CD79C46805FA02F22243C260013325
:10237400102BC5D1BDE8F0814FF6FF730360002335
:10238400037143718371C3717047036919420CBFB0
:102394000020012070470AB10183704741837047D0
:1023A40001F00703C90800EB810010B59B00046A23
:1023B4000F21994024EA01010162016A9A40114304
:1023C400016210BD08B5134B984207D14FF40010B9
:1023D400012100F0C3F94FF4001014E00E4B9842B1
:1023E40007D14FF48000012100F0B8F94FF48000C8
:1023F40009E00A4B98420BD14FF40000012100F090
:10240400ADF94FF400000021BDE8084000F0A6B982
:1024140008BD00BF0054004000580040005C00406C
:10242400F0B585B004468688324F68460D4600F004
:10243400FDF802982A68304B26F03F063604B0FBBC
:10244400F7F7360C1FFA87FC4CEA0606A6802188AB
:1024540021F001010904090C9A4221800DD853008E
:10246400B0FBF3F39BB20CF1010C032B1FFA8CFCB1
:1024740098BF0423A4F820C022E0E9884BF6FF7338
:10248400994205D102EB4202B0FBF2F39BB206E0A3
:1024940019235343B0FBF3F39BB243F48043C3F3D8
:1024A4000B020AB943F001034FF4967257434FF4F9
:1024B4007A7297FBF2F70137BFB243F400432784E3
:1024C400A38323886989AA889BB243F001032380EC
:1024D400238823F4816323F002031B040A431B0CA7
:1024E40013439BB223802A89AB8913439BB2238174
:1024F40005B0F0BD40420F00A086010041F28833D0
:102504000360002383804BF6FF72038143814FF401
:102514008043C28083817047038819B19BB243F022
:10252400010303E023F001031B041B0C0380704729
:10253400038819B19BB243F4806303E023F48063FE
:102544001B041B0C03807047828A008B92B221F01B
:102554007F4342EA00401840431A584258417047AA
:10256400014B1860704700BF00300040014B5860B9
:10257400704700BF00300040014B9860704700BFB7
:1025840000300040024B4AF6AA221A60704700BF8E
:1025940000300040024B4CF6CC421A60704700BF3A
:1025A40000300040014B1860704700BF20000E420D
:1025B400034B5B6818420CBF00200120704700BF2A
:1025C40000700040B0F5402F054B04D01A6842EA71
:1025D4008000186070475A6842F440225A6070477D
:1025E400007000400E4B1A6842F001021A6000228B
:1025F4009A60196821F0A85121F410211960094941
:1026040059600949C3F8841001F18061C3F8881046
:10261400196821F480211960DA60C3F88C207047AE
:102624000038024010300024003000201D4B9A680E
:1026340002F00C02042A10B503D0082A03D01A4B66
:1026440018E01A4B16E059685A6811F4800F59685B
:1026540014BF164B144B02F03F02B3FBF2F3114AC2
:102664005268C2F30142C1F3881101324B43520054
:10267400B3FBF2F30B4903608B680D4AC3F30313F6
:10268400D45C0368E34043608C68C4F38224145D23
:1026940023FA04F484608968C1F34231525CD34064
:1026A400C36010BD003802400024F40040787D016E
:1026B40001000020044B1A6B09B1104301E022EA27
:1026C40000001863704700BF00380240044B9A6B47
:1026D40009B1104301E022EA00009863704700BF8B
:1026E40000380240044B1A6C09B1104301E022EA9D
:1026F40000001864704700BF00380240044B5A6C55
:1027040009B1104301E022EA00005864704700BF99
:1027140000380240044B1A6909B1104301E022EA6F
:1027240000001861704700BF00380240044B5A692A
:1027340009B1104301E022EA00005861704700BF6C
:1027440000380240044B9A6909B1104301E022EABF
:1027540000009861704700BF00380240044B1A6AB9
:1027640009B1104301E022EA00001862704700BF7B
:1027740000380240044B5A6A09B1104301E022EACE
:1027840000005862704700BF003802404309012B23
:10279400074A01D1136803E0022B0CBF136F536F78
:1027A40000F01F0023FA00F000F00100704700BFA2
:1027B4000038024082B000230193054B0193019B32
:1027C40003EB80000190019B196002B0704700BFC9
:1027D4005028004082B000230193054B0193019BD4
:1027E40003EB80000190019B186802B0704700BFA2
:1027F4005028004008B5254B984207D14FF480502B
:102804000121FFF7B7FF4FF4805039E0204B984285
:1028140007D14FF480400121FFF7A0FF4FF480401F
:1028240009E01C4B98420BD14FF400400121FFF703
:1028340095FF4FF400400021BDE80840FFF78EBF2C
:10284400154B984207D14FF400500121FFF792FF36
:102854004FF4005014E0114B984207D14FF480100C
:102864000121FFF787FF4FF4801009E00C4B9842D9
:102874000BD14FF400100121FFF77CFF4FF400103F
:102884000021BDE80840FFF775BF08BD00300140D6
:1028940000380040003C004000340140005001403A
:1028A400005401400B88028810B54C8823438C885F
:1028B4002343CC8823430C8923434C8923438C89A9
:1028C4002343CC8902F44152234313439BB2038034
:1028D400838B23F400631B041B0C83830B8A038206
:1028E40010BD0023038043808380C3800381438120
:1028F4008381C381072303827047038819B19BB284
:1029040043F0400303E023F040031B041B0C03804B
:10291400704781817047038919420CBF0020012050
:1029240070470000038ACA889BB230B523F4405331
:102934000D46134303820989AB8882890B43698955
:1029440092B20B4322F4B05222F00C029BB2134316
:102954008381838AAA899BB223F44073134385B08D
:10296400838204466846FFF761FE194B9C4203D0FC
:1029740003F580639C4201D1039B00E0029BA28982
:1029840012B2002A2A684FF01901B4BF5200920013
:102994005943B1FBF2F16423B1FBF3F212011009C4
:1029A40003FB1011A08900B2002806DAC9003231F5
:1029B400B1FBF3F303F0070305E009013231B1FB86
:1029C400F3F303F00F031A4392B2228105B030BD32
:1029D40000100140838919B19BB243F4005303E012
:1029E40023F400531B041B0C83817047C1F30801BB
:1029F40081807047038819420CBF00200120704772
:102A040010B50023934203D0CC5CC4540133F9E7DE
:102A140010BD02440346934202D003F8011BFAE7B7
:102A24007047FF004C6174746963650069434563D2
:102A34007562653220323031342E31322E323730E5
:102A4400353200506172743A206943453430554C34
:102A5400314B2D434D33364100446174653A204D6A
:102A6400617920313120323031352031393A3139F0
:102A74003A35350000FF7EAA997E51000105920087
:102A84002062016F820000720070110001010000D9
:102A940000000000000000000010000080000000A2
:102AA40000000200000000008000000000000000A0
:102AB4000000010000080000000000000000000009
:102AC40000000000000000200000000000000000E2
:102AD40000003400020000000000000000000000BC
:102AE40002000000000000000000000000000000E0
:102AF4000000000000000000400000000000010091
:102B04000000000040000000000000000000000081
:102B140000040000000000000000000000000000AD
:102B2400000000000000000580000000000000001C
:102B3400000000030000000000000000000000008E
:102B44000000000000000000000000000000000081
:102B540000000000800000000000020000000400EB
:102B640080000002000000000000000000080000D7
:102B74000000000000000000000000000000000051
:102B84000000000000010000000000000C00000331
:102B9400000300000000000000000000000000101E
:102BA4000000000000000000000000000000000021
:102BB4000000000000000000000000000000000011
:102BC4000000000000000000000000000000000001
:102BD40000000000000000000000000000000000F1
:102BE40000000000000000000000000000000000E1
:102BF4000000000000000000005800000000000079
:102C040000000000000000000000000000000200BE
:102C1400000000000E080000000002000000000098
:102C24000000000000000000202000000000000060
:102C34000000000000000000000000000000000090
:102C44000000000000000000000000000000000080
:102C54000000000000000000000000000000000070
:102C6400000000000000000000000001000000005F
:102C7400000003000000000100000000000000004C
:102C84000000000000100000000000000000000030
:102C940000000000000080000003000000000000AD
:102CA4000300800000030000000000000000000892
:102CB4000000002C000000000000000000000000E4
:102CC40000000000000000000000000000001800E8
:102CD4000000000200000000000000000000007876
:102CE40000100000000000000000000000000000D0
:102CF4000000400000000000000000000000400050
:102D040000010000000000000000000400000000BA
:102D140000000000000000000000000000000000AF
:102D2400000001000000000000000000000001009D
:102D34000000000000000000000000081000000077
:102D440000000000000000000000000000008005FA
:102D5400800000000000000000008000000000006F
:102D64000000000000000008003000000000000027
:102D740000000C3020008000000000000014280037
:102D840000000000781800000020735A08000000BA
:102D940000030002000000001DDF0C000000000022
:102DA4000C30000000000000000000366C00000041
:102DB400004008FB0000001C025C000080000000D2
:102DC4002C000000000000E0F100000000000C30C6
:102DD40020000000000000000000000000002800A7
:102DE4003808000000000058080000000007000236
:102DF40000A000001C8F0C00000000000C3000003C
:102E0400000000000000003400000000200008075B
:102E14000000003C3F490000010000003C0000802D
:102E240000000000F110000000000C302000000041
:102E3400000000000200000000001000000000007C
:102E44002004017C00020000008300020000000650
:102E5400168F0E00000000000C300000000000007F
:102E640000000000000000001000700B0000003C97
:102E74003D50020000000100B80000000000000006
:102E8400F000000000000C302000000000000000F2
:102E9400001400000000000000E80000000006DE4E
:102EA4003C0200000003840200000266548F0C0000
:102EB400000000000C3000000000000000000002D0
:102EC4002C00000000000001000000243BF038004A
:102ED400000500003C00000003C20200F1000000F5
:102EE40000000C3020000000000000000000000082
:102EF4000000000001E00000002002FE500000007D
:102F0400D9A38002000000001E8F0E1000000000F4
:102F14000C30000000000000000000000000000071
:102F2400001070E30100003C27E000000000B00046
:102F34003000000000000000F000000000000C3031
:102F4400200000000000000000000000000000005D
:102F5400800000000000280000000000D9B38002B7
:102F6400000041C0168F0E00000000000C3000006D
:102F7400000000000000000000000000000030E736
:102F84002000000000000000000050A080000000AD
:102F940000200000F010000000000C3020000000B1
:102FA4000000000000000048E00000007000040081
:102FB4000000000000000000101380020000026006
:102FC400168F0E00000000000C30000010000000FE
:102FD400000000000258F000000038072C00000038
:102FE40000000000000008A0B8000000004002003B
:102FF400F000000000000C30200000000000000081
:1030040000000378A50230000000000000206C00DE
:1030140000000000001023C000C003C01685560045
:10302400000000000C300000000000000000000060
:10303400034052201000700B2800000C38000000E0
:10304400000000C003C00000A060020550000000A2
:1030540000000C3020000000000000000000014CC3
:10306400F0C000C000000000003C284E0F800000AB
:1030740000C38002000000029C05A80000000000BC
:103084000C3000000000000000000000001F0F20B2
:10309400014000900000000400080F000000000040
:1030A40000000800004294DA5000000000000C30D8
:1030B400200000000000000A000001C8F0C0004029
:1030C4000400000A000005CC0F8000000007800205
:1030D400000001429C80F800000000000C30000059
:1030E400000000000008000000000F200040000065
:1030F400000800142C1F0F0000000000B80000009E
:10310400094281F0F000000000000C3020000000B3
:103114000000000000206548F0C01001000000001D
:10312400001C055E0F80000030058002000001468F
:103134005480F800000000000C3000000000000083
:103144000000000420200F20100000000000000CEC
:10315400202A0F00000000003800000000020300D5
:10316400F000000000000C3020000000000000000F
:1031740000060148F0C0000000000000000601DC69
:103184000F80000000070402000000601580F800B2
:10319400000000000C3000000000000000000000EF
:1031A40000200F2000000000000000003C300F0051
:1031B40000009000A800000000000200F0000000E1
:1031C40000000C302000000000000000000031E886
:1031D400F0C0000000000010002001C15A8000006F
:1031E40000058402000000001F80F80000000000B9
:1031F4000C300000000000000000000000000F2060
:10320400000000000000001C3CECA50000000000D1
:10321400380000000002C080F000000000000C3004
:10322400200000000000000010000168F0D0004001
:1032340000000000102001780F80000078150402BF
:10324400000101401790F800000000000C3000005D
:10325400000000000000000000000F00000000005B
:10326400000000043C100F00000000802800000053
:10327400002001C0F000000000000C30200000001D
:1032840000000000000631E8555000000000000076
:10329400000661EA0F80000079E17C3E00000260D4
:1032A4001F80F800000000000C3000000000000047
:1032B4000000000000205500002800000000003C31
:1032C40028200F0000005900F43C00010042C30014
:1032D400F000000000000C30200000000000000C92
:1032E4000020040000000000000000000000066848
:1032F4000840800079E023C000000200408F0200F3
:10330400000000000C300000000000000008100461
:1033140020000000000000000000003C23490500DC
:10332400400008A003C000000042000F000000009D
:1033340000000C30201020007A3C20000000001C0B
:10334400F040000000180000000000000000000031
:103354000003F954000000662FC5F00000000000CF
:103364000C30000000000803C09000002C10F00195
:10337400004000F70000000000000000000000B062
:10338400C154000000003D05F000000000000C30B6
:1033940020000000323C200A001E0200A540280044
:1033A4000008000A0000000000002800000379FC67
:1033B40008A001E681AF0400000000000C3000000A
:1033C40000000003C048000000405A012000F0073C
:1033D40000080000000000002000F003C2FC02808E
:1033E4000342C00F0000000000000C302000000069
:1033F4003A3C204C0000281CF0401010001000043F
:1034040000003800000010008083FE0420C041400A
:1034140000000000000000000C3000000000000369
:10342400C00000344000F001102000CF000C080060
:103434000000000030001189FD0000C0036000009E
:103444000000000000000C3020000000323C20008E
:1034540000140008F040000000000000000000001C
:103464000000000000017A002008004781AF04003A
:10347400000000000C30000000000803C00000360B
:103484000010F00000000007000000000000000031
:1034940000000007EA0000041424010F00000000EB
:1034A40000000C3020000800723C20000000000ADC
:1034B400F0400000008000100000001EF0400000FA
:1034C40038052DFC00000000018F040000000000FE
:1034D4000C3000000B0A0003C00000000000F000E4
:1034E4000000F1BB020004000000F00000000889A5
:1034F400BEFC2000A000000F0000000000000C3003
:1035040020040100723C2000100E380AF0400040F4
:1035140000000000100020000000004001817A80BB
:103524000001426635800000000000000C300000FD
:1035340000800803C00000020010F0000000000D2D
:103544003C0000340000000000000005C000200022
:10355400004025A10000000000000C302004000AF7
:103564007A3C20001000001AF040000000A0040083
:103574000000001CF04000000000000000001407E0
:1035840001CC0220000000000C3000040500000300
:10359400C00010000000F0000000D1F33C00000067
:1035A4000010F00000001000000000000800010CF2
:1035B4000008000000000C30200005007A3C2000C8
:1035C4000000001AF040100050A004000020001C6D
:1035D400F060000001A063C10000100707C0801064
:1035E400000000000C300000050E0003C0001000B5
:1035F4000000F0001000D9BB3C0000240000F000E3
:10360400000000A003C00400000424800080000027
:1036140000000000000000007A3C200000262A5B25
:103624004240004000000000001C00ED5A0000046D
:1036340001E000000002000000AF040000000000F0
:103644000000000000000803C1000014024CE20066
:10365400404000000000000001CC1A010000F0907E
:10366400000000040000010F000000000000000042
:10367400028005007A3C200A001E7078AF100040DA
:103684000000000A0020006AA500280000A7EA0044
:1036940000A00000418F04000000000000000200B0
:1036A40000800803C008003E2020AF100040000046
:1036B40000080004015055002000000F6C00008039
:1036C4000003810F00000000000000000300000060
:1036D4001A15400C0016024C304230000000000461
:1036E4004020396AA00010000193382800400003EC
:1036F400C0000000000000000000000000000015F1
:10370400400400000270B10090000000000C00347E
:103714006370F50010000080002820C06003C00022
:1037240000000000000000000000000007BC1000C2
:103734000014287B4240000000000000000000FC50
:103744000E02000000F5F8000800E0000000000090
:1037540000000000000000000000043C00200014F1
:10376400286CD100800000000000001428D00F0055
:10377400000000FF810000000000000000000000C5
:10378400000000000000000007BC10000000625BA5
:1037940042400000001000002014000AF040000025
:1037A4005801FA010800000000EF040000000000C6
:1037B400000000000000043C08000000665DE20018
:1037C400800000F00200E0000000F00000000000B3
:1037D400C20000000000010F000000000000000013
:1037E40000000000802950040026647B4240000051
:1037F40000000000863604000000000000012C8157
:1038040000000000000000000000000000000000B4
:103814000000101680040026647DD10080000000A2
:103824000000001428000000000000097C000000D3
:103834000400000000000000000000000000000080
:103844000000000000000258424040000000000058
:103854002006005AF50000008005F805000000006D
:10386400200A5400000000000000000000000000D6
:10387400000000000248E200000000000000000018
:103884000340A000000050C1EC00000000021C0531
:10389400A0000000000000000000001B0000000069
:1038A40000000159014040000000000080000000B9
:1038B400000000007810000000000040000000003C
:1038C4000000000000000000000A000000000000EA
:1038D4000059A7000000000000000E0000000000D6
:1038E400000008A00000000000000000000000002C
:1038F4000000000000000180000000000000014AF8
:10390400F0D000000008000000002E1CB1000102ED
:10391400001869550000000240000000000000008B
:1039240000000000008A0000000000002C190F00B5
:10393400044000070000000038DF7200028000D954
:1039440042A800080007400000000000000000003A
:103954000280050076A8000A000001C8F0C0280013
:103964000008000A002003FCAF2328007818029501
:1039740000B401E017CAF4000000000000000200D7
:103984000100F4000008000000000F002000000700
:103994000008201C0150DF00200008C101680082DB
:1039A40000201700A1000000000000000300001F19
:1039B4003F99C480002061C8F0C0100000C0000C12
:1039C400001E001CF040300050A03BC1804203C7E1
:1039D4009DCA50000000000000000300000DD03F0D
:1039E400C00000042C200F003000310F000C000038
:1039F4000000F000100000A043C0004401E43505BD
:103A040051000000000000000100001A1B191A10E8
:103A140000060148F0E001000000000001200268F7
:103A2400A50000800010000000000167BDEA02004C
:103A34000000000000000100001032160200000027
:103A440000200F0002000007000000042B50550066
:103A5400010000900000000000202E0F5000000024
:103A6400000000000000010012DD1000000001E869
:103A7400F0C0000080900000000005EE200201006C
:103A8400000DE005000A01668E8A020000000000B5
:103A9400000000000108B6140A40000000000F00F6
:103AA4000020709B0000000020202000028000897C
:103AB400AC0000040002EF0FA000000000000000B2
:103AC400000005801640500000000168F0C00000AE
:103AD40080000000000466CEA5000000000D628195
:103AE4000000000716AA50000000000000000000BB
:103AF40001001A29C860000000000F000000300512
:103B04003C000E3620F055000000000D400000007F
:103B140000073C0AA00000000000000000000D8F18
:103B240093DD1600000605E855400000819004006E
:103B3400006039E87002000030057A0100000807CF
:103B44004D8A000000000000000000000D1A32142D
:103B54000020000020205500000091E33C00009468
:103B64000150F00000000099F80000080346D40F4B
:103B74005000000000000000000008000000000CDD
:103B84000020040000003000999004000036041C5A
:103B9400F0400001000000000000004795EA00002A
:103BA4000000000000000000050000000008000400
:103BB400200000001000999B3C000C142800F00029
:103BC400000200800000000000242D0FA00000006F
:103BD40000000000000000000000000000002000C1
:103BE40000000040000000000020054B70000000B1
:103BF40000007BC100000003B59205000000000036
:103C04000000000000000000000000004000000070
:103C140000400090000000242368F00000000080B1
:103C240043C00000000724CE000000000000000094
:103C3400000000000000000000340000000000400C
:103C44000000000A002002FABD03280001E0000081
:103C540000A00242CF81C00000000000000000006C
:103C6400000000000000002C2800000000400000BC
:103C7400000800240160FD0820000100000000800D
:103C8400006217C3C0040000000000000000000030
:103C94000000000000000208500010000000000CAA
:103CA4000020641EF0401000000063C10000020305
:103CB40025AB94000000000000000000000000009C
:103CC400000000000050A00010000000000C002CB8
:103CD4002400F0001000000043C0000000401793CF
:103CE40080800000000000000000000000000000D0
:103CF4000000000000000000000000000026064E46
:103D0400A5000000000000000000014035E8D404D4
:103D1400000000000000000000000000000000148B
:103D240000000000000000000000000625F055001F
:103D340000000000000000000002A698E00000005F
:103D4400000000000000000000000000000000006F
:103D54000000000000000000000072DCF50000001C
:103D6400000000000010016000EF040000000000EB
:103D7400000000000000000000000000000000003F
:103D8400000000000000001C00F0500000000000D3
:103D9400000000100000000F000000000000000000
:103DA40000000000000000000020000000000000EF
:103DB40000000000002066DEA500000000000000F6
:103DC40000000200018F0410000000000000000049
:103DD400000000000000003C0000000000000000A3
:103DE4000000002423D0AA0000000000000000000E
:103DF4000143C00F020000000000000000000000AA
:103E0400000000000000027B100000000000000021
:103E14000E00701A8002000000000000000A00007A
:103E240027E0540000000000000000000000000033
:103E340000000000024C2401000800000000000003
:103E44000050400000000000000000000040240A70
:103E5400000400000000000000000000000000005A
:103E64000000000000000100000000000000381CF9
:103E7400F0400000001000000000036007D40000C0
:103E8400000000000000000000000000000000002E
:103E94000000000002000000000000342400F000D4
:103EA400000000D00000000001601680000800003F
:103EB40072009011010101000000000000000000E8
:103EC400000010000000000000400000000000019D
:103ED4000000000000400002000000000000080094
:103EE40000000000000000000000000000000000CE
:103EF400200000000000008000000000000200001C
:103F040000000000000000000000000000000000AD
:103F14000800000000000000000000000000000095
:103F2400000000000000000000000000000000008D
:103F3400000000010000000000000400F000000088
:103F4400000000000000000000000000000000006D
:103F5400000000000000000000000000000000005D
:103F6400000000000000000000000000000000004D
:103F7400000000000000000000000000000000003D
:103F8400000000000000000000000000000000022B
:103F9400000C0000000008000000300000000000D9
:103FA400000000000000000000000000000000000D
:103FB40000000000000000000000000000000000FD
:103FC40000040000000000001000000000000000D9
:103FD40000000000000000000000000000000000DD
:103FE4000034000000000000000000000000000099
:103FF40000000000000000000000000000000000BD
:1040040000000000000000000000000000000000AC
:10401400000000000000000000000000000000009C
:10402400000000000000000000000000000000008C
:10403400000000000000000000000000000000007C
:104044000000000000000000000008000000000064
:10405400002000000000000000000000000000003C
:10406400000000000000000000000000000000004C
:10407400000000000000000000000000000000003C
:10408400000000000000000000000000000000002C
:1040940000000000000000000000000200000B000F
:1040A400010000000000000C0000000000000000FF
:1040B40000000000000000000000000000000000FC
:1040C4000000000000000000000100800800010062
:1040D40000020000000800000000000004000000CE
:1040E40000000000000000000000000000000000CC
:1040F40000000000000000000000000000000000BC
:1041040000000000000000000000000000000000AB
:10411400000000000000000000000000000000009B
:10412400000000000000004000000000000100004A
:10413400000000000000000000000000000000007B
:10414400000000000000000000000000000000006B
:104154000000000000000001000000000002040054
:10416400000000000000000000000000000000004B
:10417400000000000000000000000000000000003B
:1041840000000080000000000002000E000000009B
:1041940000007000000000000000000C300000006F
:1041A400000000000000000000000000000000000B
:1041B40000000000000000000000000000000000FB
:1041C400C00100F000000000000C302000000000DE
:1041D40000000000000000000000000000000000DB
:1041E40000000000000000000000000000000601C4
:1041F400C0F000000000000C3000000000000000CF
:1042040000000000000000000000000000000000AA
:10421400000000000000000000000000000000F0AA
:1042240000000000000C302000000000000000002E
:10423400000000000000000000000000000000007A
:10424400000000000000000000000001C0F00000B9
:104254000000000C3000000000000000000000001E
:10426400000000000000000000000000000000004A
:104274000000000000000001428000F00000000087
:10428400000C3020000000000000000000000000CE
:10429400000000000000000000000000000000001A
:1042A4000000000000036041C0F000000000000CAA
:1042B40030000000000000000000000000000000CA
:1042C40000000000000000000000000000000000EA
:1042D40000000000003C0AF000000000000C302048
:1042E40000000000000000000000000000000000CA
:1042F40000000000000000000000000000000000BA
:1043040000000021E5F000000000000C3000000077
:104314000000000000000000000000000000000099
:104324000000000000000000000000000000000089
:104334000000000000000000000C3020000000001D
:104344000000000000000000000000000000000069
:104354000000000000000000000000000000000059
:10436400000000000000000C30000000000000000D
:104374000000000000000000000000000000000039
:104384000000000000000000000000000000000029
:1043940000000000000C30200000000000000000BD
:1043A4000000000000000000000000000000000009
:1043B40000000000000000000000000000000000F9
:1043C4000000000C300000000000000000000000AD
:1043D40000000000000000000000000000000000D9
:1043E40000000000000000000000000000000000C9
:1043F400000C30200000000000000000000000005D
:1044040000000000000000000000000000000000A8
:104414000000000000000000000000000000000C8C
:104424003000000000000000000000000000000058
:104434000000000000000000000000000000000078
:10444400000000000000000000000000000C30200C
:104454000000000000000000000000000000000058
:104464000000000000000000000000000000000048
:1044740000000000000000000000000C30000000FC
:104484000000000000000000000000000000000028
:104494000000000000000000000000000000000018
:1044A4000000000000000000000C302000000000AC
:1044B40000000000000000000000000000000000F8
:1044C40000000000000000000000000000000000E8
:1044D400000000000000000C30000000000000009C
:1044E40000000000000000000000000000000000C8
:1044F40000000000000000000000000000000000B8
:1045040000000000000C302000000000000000004B
:104514000000000000000000000000000000000097
:104524000000000000000000000000000000000087
:104534000000000C3000000000000000000000003B
:104544000000000000000000000000000000000067
:1045540000009000000000000000000000000000C7
:10456400000C3020000000000000000000000000EB
:104574000000000000000000000000000000000037
:104584001000000000000000000000000000000C0B
:1045940030000000000000000000000000000000E7
:1045A4000000000000000000000000000000D00037
:1045B400000000000000000000000000000C30209B
:1045C40000000000000000000000000000000000E7
:1045D40000000000000000000000000010000000C7
:1045E40000000000000000000000000C300000008B
:1045F40000000000000000000000000000000000B7
:104604000000000000000000000000000000006046
:104614000000000000000000000C3020000000003A
:104624000000000000000000000000000000000086
:104634000000000000000000000000000000000076
:10464400000000000000000C30000000000000002A
:104654000000000000000000000000000000000056
:104664000000001000100000000000000000000026
:1046740000000000000C30200000000000000000DA
:104684000000000000000000000000000000000026
:104694000030008000000000000000000000000066
:1046A4000000000C300000000000000000000000CA
:1046B40000000000000000000000000000000020D6
:1046C40000000000000000000000000000000000E6
:1046D400000C30200000000000000000000000007A
:1046E400000000000000000000000000002800009E
:1046F4000000000000000000000000000000000CAA
:104704003000000000000000000000000000000075
:1047140000000000000000000000000000000B008A
:10472400143000000000000000000000000C3020E5
:104734000000000000000000000000000000000075
:104744000000000000000000000000000D214100F6
:1047540000000000000000000000000C3000000019
:10476400000000000000000040DB0000000000002A
:10477400000040034DA5008000108D80140000004F
:104784000000000000000000000C302000000000C9
:104794000000000000024E5F020000000000000064
:1047A4000000ED02400000819FA1430200000000D0
:1047B400000000000000000C3000000000000000B9
:1047C40000000403D00000000000000000014002CB
:1047D400DBF500010010098014000000002C80802B
:1047E40000000000000C3020000000000000000069
:1047F4002C785A0A00000000000000000602DAF4D7
:10480400000280980FA14300000000248B5408008C
:104814000000000C30000000000000000000040054
:10482400000000000000000000003C3CD00001003B
:1048340000000D001400000002000F000000000042
:10484400000C3020000000000000000020000000E8
:1048540000000000000000002061D80202000000F7
:104864000DA14300000000568F0800000000000C5A
:104874003000000000000000002000400050000054
:104884000000000000001E00200A000000000900D3
:10489400140200E000020F0000000000000C3020B1
:1048A40000000000000000400039D8500000000063
:1048B400000000001C00EA0A200000000FA14300D1
:1048C400000000048F0800000000000C300000000D
:1048D400000000000000003B400800000000000051
:1048E400000000316D0010000000AD801400004293
:1048F400C0000F0000000000000C30200000000089
:10490400000000000062F81802000000000000002F
:1049140000046F08000000181D2143000003400636
:104924008F08000A0000000C300010000000000096
:1049340000000002500000000000000000000424F9
:10494400000000100000898014000002C0000F0065
:1049540080040000000C3020000000000000000073
:1049640006024CA020000000000000002078000097
:10497400001000019D214300000340168F08000031
:104984000000000C3000000000000000080014309B
:104994004000000000000000080200274A850020B3
:1049A4000000AD001400800140000F000000000072
:1049B400000C30200000000000000A001E065850C1
:1049C4000000000000000A000005CC40402900005F
:1049D4001F214300A00000148F0800000000000CF9
:1049E400300000000000000000003C036A52100088
:1049F4000000000000000000E94200000000A900DF
:104A0400144A00014000000020000000000C302087
:104A1400000000000000000C0E624E7A400000000E
:104A24000000000000014B50400000000F21430033
:104A34000001C29400080000000000000000000013
:104A4400080821402000000020A0200000000000F1
:104A54000000003AEB80000138008165000000028C
:104A64004000000000000000000000000000015EA3
:104A7400A140800000014AA00000000000000000E6
:104A84000006FA00000000019764000000026000C4
:104A940000000000100000000000000000D01080A2
:104AA40040000436EDA500000000000000001C02D8
:104AB40060CB00810001077F0C000001C4000000EE
:104AC400000008000000000000000C0020448000EA
:104AD400046579A74000000000000000266AEAC3CC
:104AE40042028031C3FF4D050002638000000000D4
:104AF400000000000000000D0B9E000000000020DC
:104B0400200A0000000000000000447ACF8000006A
:104B140000090581002000024014EC4080000000E0
:104B240000000000000B0113804000100004F80A8C
:104B340001000000000000102027790008004078E0
:104B4400A128010801020017FD0400000000000074
:104B5400000000500BF4200000001C3420A02804A6
:104B64000000000000000001E0D33840007003E8BA
:104B7400000000000034C8D0000000000000000065
:104B8400002001120000800020795AA020040000B7
:104B9400000000000000EA4342000000016C200015
:104BA40000000016B814000000000000000000001F
:104BB40080DB000000001633CD240000000000005C
:104BC40000000242E00000000008B1E6900000008E
:104BD40062E4A5C0800000000000000000070A3A5B
:104BE400C04000003E004C10000000000000000126
:104BF4000E2B5C5000000050076590000003400736
:104C0400CA0600000000000000000000885B4000AD
:104C140000001676607600000000000000200434D6
:104C2400005F000000580D4294800000441D901065
:104C3400000000000000000000038857420000004C
:104C44002E74CAB1620000000000004000344E5FC0
:104C540000000050A3F3E800000202B7B000000017
:104C64000000000000000000000402800800343B43
:104C7400E01800000000000008001C22FEA50860E7
:104C84000000A5810000800343C40AC000000000A6
:104C9400000000000000003B02800A003E05DA0824
:104CA4000200000000000A000007DA405829000151
:104CB400D1280108A000035DCA0420000000000000
:104CC400000000000854140000003C21D9800000BA
:104CD4000000000000000203EB5A00000201B3E8E8
:104CE40000000000203E05A00000000000000000BD
:104CF40000018B87A80000002005CF000000000001
:104D0400000000001400EF4050000518A16E0000E0
:104D140000014606EF50000000223D080009000093
:104D2400009F000000002402CB40000000000000AF
:104D34000090003749A109000001D00000000000E4
:104D4400003CE800000000C03F800021000300F2A6
:104D5400E000000000637800000000000000000094
:104D640000026D4241003801C00000000001E0165D
:104D7400C00000000000140A000000000093E000DE
:104D840000000002C0000800000000000000804095
:104D9400F80A080040399DB31C010012C204ADD0CA
:104DA4000000000024A0000000001C3E00000000E1
:104DB4001E006C80020000000000000040796B4A75
:104DC400500000D1FDF70D0000E8406EEEF0000049
:104DD4000030000000000000003640802000004247
:104DE4004000000000000000000000027D001000F0
:104DF40000D10B4000400001E0059200040000C017
:104E040000000000040500824040001000735A02B4
:104E1400020040000000001000206C08000040392F
:104E24008BB9400001014007A006000000400000CB
:104E340000000800001C00000020027C700000003C
:104E44000000000000003C61600000000008DDF08C
:104E540000010000401504001000000000000000E4
:104E640010001C1B200080401C235CA000000000DC
:104E7400000000000E75FAA0400000100FBC208056
:104E84000002000EA000200000000000000000004E
:104E940000500140000014796E0000000000000082
:104EA40000003C60000000000058876430000001EE
:104EB400603C0A00000000400000000000039C5F0A
:104EC400800800002E3C4F08200000000000000075
:104ED40000280000000002B9B5EC200000034604DD
:104EE400C000000002400E8FA00028018054000082
:104EF4000000363760000000000000000000822E31
:104F0400703C080000008780D000000366CDEC8070
:104F1400100002001FDE7080138B9E3E200080A0D4
:104F24003E06DA80020000000000020754017C7C87
:104F3400530000001568F50A000142B4FD040000A6
:104F44000343400000020009905C140000000C417F
:104F54006B0000000000000008013428F058002015
:104F64000001094014008003601E840080000200D8
:104F74004000000280070E168000000036704F02C9
:104F84000000000000000A00A0616E18022805005D
:104F940088782800A0014015981000000020000027
:104FA400000000050E0003C04000002BDA003100B1
:104FB400000000000000803ED00A000100000B0049
:104FC40000000002E41CCC801000C060000000005F
:104FD4000000010283D200000002D8040000000097
:104FE4000000000140281A0500408010013028000C
:104FF40000014295AC24000000623D000100000065
:1050040009DC3CC0000CA425FD8000010000000068
:1050140001001C227A01200400909782940000026F
:10502400C380000000000040358050100000091BC0
:105034003DC080016006CB0010028000000000002B
:1050440020066F07600000819FE1652800020000D0
:105054000000000000220D000280204F8098000014
:1050640000000063EA0020000000000001002C039F
:10507400D0E300000000E5000C000000000100F097
:10508400000001C03EE80030000B887EA0008000D4
:10509400006459400001280000000107A0206AC3F1
:1050A4006300007811B0080800000000C0F500009B
:1050B40000420300A00000000CD4000010001C7685
:1050C400700000000000000000003E3CFF030000F0
:1050D4000071BB801400000000000000000002000A
:1050E4000FA0A00000000097008E800020605A806E
:1050F40012000000000000002E7E4F02000000009D
:10510400AB3168000000000000000000014006E030
:10511400000000030AF40000000002241050000004
:10512400000000000000023EC800000000F1DDF8AD
:1051340000811000034000000000E36015B020006F
:105144000000089202800000063C7E50000000002F
:10515400000000001E02DE80000000D9DF320100E2
:10516400000007C00000000002440CA00000000D75
:105174000A5600000001027C00000000000000004C
:1051840000003C015E5B000000F100000000001024
:10519400001E8000880002021CC801000008001FD5
:1051A400A00000001C7000000000000000000000CF
:1051B4002000EEA540000001E00000000008C0252A
:1051C400A806100001624600000000050A1B5000FA
:1051D4000000343AD0E3010000000000000004267F
:1051E400E000000000010BF00000000000000000DF
:1051F4000000006066C2002003800113C0000000AC
:10520400006F5AC352000000000000002000ECA010
:1052140000000830CFE40840000000000000000057
:1052240003424505F000000B0BB402881800BC02D1
:10523400DF0300000000000008000069D0C3112053
:10524400005005F7FC00800002E7F0200000020295
:10525400C08AF0000008003380000A071C00FC022A
:105264000000000000000A001E70EEC7422800B1D2
:10527400ADA1FD20A000000D9000000002434000FD
:10528400000000070BF780003001002BD80000005D
:105294000800000000001C27C92500000000CDF410
:1052A4000060000027400000000003C04000000030
:1052B40000050A9200800000803CCB08100000002A
:1052C4000000002006005C000000000001FC20003B
:1052D4000001E2C00000001000002600500300009E
:1052E40008B0294041002E640000000002000000C4
:1052F4000000AC7C0000000080000B3108040000BA
:10530400000200A0001000002F800003000581802F
:1053140016944100262C000000000000000000004C
:105324007C20000000010000000605420000000F80
:10533400C0A480000142830020800001000C25806D
:1053440000003401D0A020000400000000001E4230
:10535400E0AF21000000804280020003C0010A0087
:105364001400000044A020300009803FA5905000A4
:1053740000721E5000000000000000003C72EEA508
:105384004000007013B280000000500C8A05000039
:105394000142BC00000000000000000000000441C5
:1053A400F0FF20000000000000001C216B10000032
:1053B4000008000000000A01C7DE8FF0840002002C
:1053C4004EC0A00000001800000000001C637EF71F
:1053D4000200000000000000206DFC0000000071CD
:1053E4008000000004020786E7F50000014004087D
:1053F400020000000000154000003E40E0C3000031
:105404000000800100000C00601A00000000000190
:105414006802182023800FF0840003402CE0012050
:105424000000005A15500002B472DCE302000400CC
:1054340000000040006BF85A02000018E101680007
:10544400100142000FF100000000340010100001B0
:10545400000803C0100E006F40E500003A00000091
:105464000000000030A000000200CD810800100000
:10547400040590019000000000C022240008001AD6
:105484003C380000003F4CA5020000000000000072
:1054940000006EA0000004000D3B8D881000021C6B
:1054A400D014000000024F0000000000080803C0F0
:1054B40000000203C8000010000000000000243CAB
:1054C400000000000000008140000000002682006F
:1054D4000C0020007C850000000001523C30000CD0
:1054E4001669CD8000308000000000280000000014
:1054F40000000000C3B140000000000D9344000010
:10550400024424B0000200000F0003C040003C2A03
:10551400F80408004000000008423C7DC000002060
:1055240000000FAF6840800267C6D5810000020604
:1055340005840002800001723C30200020066A00CD
:105544000000400000000A00062FDE0212280000BE
:10555400053E0564A0026216F984800000440DC073
:1055640042000000000003C14000000000000000F1
:105574004000000000804002FC0000010008000020
:1055840000000A00020000000000006624E002009F
:10559400000000723C3020041600000000004000AF
:1055A400000000008002D808000200500000000043
:1055B400000146400000000001400000000300011B
:1055C400000803C0100800400000001000000B2475
:1055D4000800000000000000021080815400000058
:1055E400000200A00000000000000003000D187A73
:1055F4003C306000002800000010000000040C0093
:10560400000000000030008015A1550000000005D6
:10561400C0A000000142800000000000000803C098
:105624001000000000000000000001300000002015
:1056340000000000000000803C00000023E5D000D2
:1056440010000006800000000001805A3C30600019
:1056540000000000000000300004004A00040000C4
:105664000000001807A3C30000014077C800000031
:105674000000000000000280000003C010000021B0
:105684007C00010000700D240000000000000001F7
:10569400200000003C0000014436004000000000EF
:1056A400000000000000005A3C3060000073FC4021
:1056B40000000080080000000000000000028000DC
:1056C40005A3C300006203B7A00020000002BCD001
:1056D40082000000000003C010001C2C0000000029
:1056E400000109000000004000000000000000006C
:1056F4003C00000007870050000000005EE000004E
:105704000000007A3C3040002E0000000000000041
:1057140088000002003800000000000007A3C30056
:105724000001E764AFA000000000000000000000DA
:10573400080803C05000142B500000000001BD00F5
:1057440000000000000000000000E0803C000202B5
:1057540042A5B0F0000000000000000000018152EA
:105764003C30002036077E0A300000009000000024
:1057740000000000000000199523C300040166D452
:10578400A0B000000000000000000000080803C0F2
:105794004000000020A000102000E70000000400EA
:1057A4003050A000001080803C000000029C005299
:1057B4001000000000000000000019523C320000FC
:1057C400000178A000100000100000002000CE505E
:1057D400400000819523C30000016756C8B0A800AB
:1057E40000003FE0011200001B0003C01000000293
:1057F400D000002000F8F10008000002E0A580209D
:105804000000E0003C00000543430A0014000000CF
:105814000CF1000280000A723C3020001602C8809D
:1058240022A80071E8000A080000400060288000F7
:105834001723C30000020006CA0000000400000091
:1058440000000000000A400001020023CD00000017
:105854004011FD000000003C205090000000006456
:105864003C00000002C30500080000000000000026
:10587400000000184020010016065A100000000025
:10588400F80000000004CA5040000000056FC30087
:105894000000069CC50100000072007011020101A5
:1058A40000000000000000000200000000000008EA
:1058B40000000000020000000000000800000000DA
:1058C4000000200000000000008000000000000034
:1058D40000000000000001000000000000040000BF
:1058E40000000100000000000000000000000000B3
:1058F4001000000000000000000000000000000094
:105904000000000000000000020000000000000889
:105914000000000000000000000000000000000083
:105924000000000000000000000000000000000073
:105934000000000000000000000000000000000063
:105944000000000000000000000000000000000053
:105954000000000000000000000000000000000043
:105964000000000000000000000000000000000033
:105974000000000000000000000000000000000023
:105984000000000000000000000000000000000013
:105994000000000000000000000000000000000003
:1059A40000000000000000000000000000000000F3
:1059B4000000000000000000000000000000800063
:1059C40000000000032000000000000000000000B0
:1059D40000000000000000000000000000000000C3
:1059E4000000000000000000000000002000000093
:1059F400000000000000000000000000000000069D
:105A04008000000000000000000000000000000012
:105A140000000000000000000000C00000000000C2
:105A24000100000000000000000000000000000071
:105A34000000000000000000000000000000000062
:105A44000000000000000000000000000000000052
:105A54000000000000000000000000000000000042
:105A64000000000000000000003000000000000002
:105A74000000000000000000000000000000000022
:105A84000000000000000002000000000000000010
:105A940000000000003000000000000000000000D2
:105AA40000000000000000000000000000000000F2
:105AB40000000000000100000004000000000000DD
:105AC4000000002000000040000000000000000072
:105AD4000000000000000001800000000000000041
:105AE40000000000000000000000000000000000B2
:105AF40000000000000000000000000000000000A2
:105B0400000002000000000000000000000000008F
:105B14000000000000080000000000000000000079
:105B24000000008000000000000000000000800071
:105B3400020000000000000000000000000000005F
:105B4400020000000000000000000000000020002F
:105B54000000000000000000000000000000000041
:105B64000000000000000000000000000000000031
:105B740000040000000000000000000000000040DD
:105B84001030C00000000000000000000000000011
:105B94000000000000000000000000000000000001
:105BA40000000000000000000000000000000030C1
:105BB400C000000000000000000000000000000021
:105BC40000000000000000000000000000000000D1
:105BD4000000000000000000000000001030C000C1
:105BE40000000000000000000000000000000000B1
:105BF40000000000000000000000800140000000E0
:105C0400000000000000000000000030C0000000A0
:105C14000000000000000000000000000000000080
:105C24000000000000000000000040000000000030
:105C340000000000000000001030C0000000000060
:105C44000000000000000000000000000000000050
:105C54000000000000780000800000000000000048
:105C64000000000000000030C00000000000000040
:105C74000000000000000000000000000000000020
:105C8400000000080000C000000000000000000048
:105C9400000000001030C000000000000000000000
:105CA4000080000000000000000000000000000070
:105CB40000000000000000000010000000000000D0
:105CC40000000030C00000000000000000000000E0
:105CD4000000000000800000000000000000000040
:105CE4000000000000000028000000000000000088
:105CF4001030C000000000000000000000000000A0
:105D0400000000000000000000000000000000008F
:105D140080000000000000000000000000002030AF
:105D2400C0000000000000000000000000000000AF
:105D3400008000000000000000000000000080005F
:105D44000000000010000000000000001030C0003F
:105D5400000000000000000000000000000000003F
:105D6400000000000000000000001000000000001F
:105D7400000000000000000000000030C00000002F
:105D8400000000000000000000000000000000000F
:105D940000000200000000D0D0000000000000005D
:105DA40000000000000000001030C00000000000EF
:105DB40000000000000000000000000000000000DF
:105DC40000000000000000000000000000000000CF
:105DD4000000000000000030C000000000000000CF
:105DE40000000000000000000000000000000000AF
:105DF400000000000000000000000000000000009F
:105E0400000000001030C00000000000000000008E
:105E14000000000000000000000000000000081264
:105E2400FD800000084000000000000000000000A9
:105E340000000030C000000000000000000000006E
:105E440000000000000000000000000A02B45FD05F
:105E5400000000000000000000000000000000003E
:105E64001030C0000000000000000000000000002E
:105E74000000000000000000000008135C59B0009E
:105E84000010F13800000000C3D6A000000000306C
:105E9400C00000000000000000000000000000003E
:105EA4000000000000000000017A48D0A000040FA8
:105EB4000000000000003C14000000001030C0008E
:105EC40000000000000000000000000000000000CE
:105ED4000000000000000B886B59A0014010F1384D
:105EE40060000000C3C4E00000140030C0000000E3
:105EF400000000000000000000000000000000009E
:105F04000000000002046C10B000400F00002000EC
:105F140000003C00000000041030C000000000003D
:105F2400000000000000000000000000000000006D
:105F340000000A92EAD0A000C010F138000000006E
:105F4400C3C4A98F00000030C0000000000000009E
:105F5400000000000000000000000000000000003D
:105F640002A25959B000800F0040000000003C011B
:105F7400010800001030C000000000000000000014
:105F840000000000000000000000000000000B887A
:105F94006B50B0000010F13800000000C3C4A0181A
:105FA40000000030C00000000000000000000000FD
:105FB40000000000000000000000000002067C0950
:105FC400A000000F0040000000803C01000E000013
:105FD4001030C000000000000000000000000000BD
:105FE400000000000000000000000A92FB80000096
:105FF4000010F17800000000C3C5E000000000308C
:10600400C0000000000000000000000000000000CC
:10601400000000000000000002A248700000000F11
:106024000000000000003C00000000001030C00030
:10603400000000000000000000000000000000005C
:106044000000000000000B8A7B01A0208010F17A80
:1060540000000000C3C5A00002000030C000000022
:10606400000000000000000000000000000000002C
:106074000000000002046C010000800F00014000D9
:1060840000003C00000000001030C00000000000D0
:1060940000000000000000000000000000000000FC
:1060A40000000A92F90000000010F16366C00000CD
:1060B400AA85E01810000030C000000000000000B5
:1060C40000000000000000000000000000000000CC
:1060D40002A25B000020000F0041428000002A81E0
:1060E400000000001030C0000000000000000000AC
:1060F400000000000000000000000000000000009C
:10610400000000000010F17006C00000000008014B
:10611400000C0030C000000000000000000000007F
:10612400000000000000000000000000000000006B
:106134000000000F0040028000000000010802047B
:106144001030C000000000007E7EA0000000083C6B
:10615400C0100000000060000000083D4000000086
:106164000010F12800000000908D800A000000302B
:10617400C0000000000042BAFC000004003C200003
:10618400000000036C000800003C00000000020F47
:1061940000000000000122CFF10A00001030C0000E
:1061A400000040005F32F4602050083D60000001B0
:1061B40040005C000050083D40000009400AA1284E
:1061C40000000500A93CC10A00140030C000000012
:1061D4000000FF0E86000012003C00000000400298
:1061E40040000010003C00500014400AA0000007CA
:1061F40001011527C50000041030C0000000000094
:106204000E9E56000024083DC0700000800040002F
:106214000020083D4050A000C02A500006C00301E1
:106224001406110000080030C000000000000FDA5E
:1062340040000020003C00080014C003800000203F
:10624400003C2050A0000005A02802800000280285
:10625400D580140C1030DC0000000040CC50460403
:106264000004083D60108000000040000000083D6C
:106274004080A1C0002A500000000000015DC00A57
:1062840000000030C00000000000CC0B002800001B
:10629400003C20090000000380000000003C203086
:1062A400A0000005A028000000800001F00A000002
:1062B4001030CC001E000000000020700002083CDA
:1062C40040100040000000000000083D6000002075
:1062D400000000000000000001548D9B12000030FB
:1062E400C00000000000000004000000003C200882
:1062F40000000003C0000100003C0000000000009A
:106304000000000000000142050A00001030C00037
:1063140000A200020F7000283800000000000020D6
:106324000000207C0800083D600000200000000000
:10633400000080300016980002000030C000000009
:1063440000040F003C405000000000000000000367
:10635400E43C0000003C00000000000000000007D6
:1063640000000801AD0040001030C0001E00020211
:106374000F30007000000000000010000080266450
:106384000000083D600000200000000000008020A4
:106394001287B90A01480030C000000200000F0053
:1063A4000040000000000000D01000F3A66470005C
:1063B400403C2000000000000000000080002D642C
:1063C4009B0002481030C000000000820F3800001B
:1063D400000000000000000000801E640030083C43
:1063E400600001C0000000000000000000468000C2
:1063F40000000030C000000000000F08340030002E
:10640400000000000020003380640020003C2000D5
:1064140000000000000000000001003680000000C1
:10642400004021E000000000551A766800082C3D69
:10643400CA000000000000000800083DE0980000C9
:10644400102831FE06000000A81CA0000000000077
:10645400050000000200AA025400000003C0C000AE
:106464000000000000000000003C20100000000EAE
:1064740033A143C00000ABC2E000800000400180B3
:10648400000000000000002802002C3C4E00000127
:10649400400000000800083CC0001009106831F5F5
:1064A400C0000500AA9C0000001000000D030C4071
:1064B400000000001400040003C0000000004000BD
:1064C40000000000003C00008010400E316423C036
:1064D40001009540F0000004004020A000000000EE
:1064E4005012460000082C3C4A98100002001C0080
:1064F4000020083CC0000000C000000006D20000DC
:10650400BC1C00010000000014000D000000000A83
:106514008000000003C01010800000000000003064
:10652400003C00000000C000000002800000BC022B
:1065340000080000004021C01B0000005076546C8D
:1065440000081C3C4A019000000000000000083CC8
:10655400400000080000A5A1E004000000000000C5
:10656400000000000D000B000000F00600280000F1
:1065740003C01000E000000000000000003C200008
:1065840000100900A08000000000000000000000CE
:10659400004021A99D0000446610406000002C3C8E
:1065A4005E001000000000000000083C4001900064
:1065B4000000000002C41000000000000000000001
:1065C4001C0799000000990AC040000003C00000A5
:1065D400F000000000000000003C200080020000E9
:1065E400000002002000000000000000004000C87D
:1065F4001E000000C61A400000001C3C5A000000A7
:10660400000000000000083C600181C000000000A0
:106614000000000000000000000000002D0F00003A
:106624000000C93E0000000013C000000044000048
:1066340000000000003C0000000000000002C00058
:106644000000000000094000004001E018000200C2
:10665400815BE06000000AA85A019000000000007D
:106664000000083CE07000000800A37C000000006B
:1066740000000818000000000C0010000000BDD647
:10668400E440000012A80000F00001000000000037
:10669400003C000800000000007C00000000000036
:1066A40001000000004000E81D4000005A7680010F
:1066B4000000000000001000C00000000000000006
:1066C40000000000000FA1294000030000000000AA
:1066D400000C000000090E200000A007C00080008C
:1066E400000000008000400000000000000000F0F6
:1066F4000214004FF0A94348000000000000000805
:106704000003C4001B0000005A3754040000083D75
:10671400E0000000000000000000183CC050A00091
:10672400002B5BB000400000A940000100000803FA
:10673400C00008000000500B16207002003C00004E
:106744000000000000000002203C0050A00000A156
:10675400A5A00206000016808D0E000000000000B7
:106764001E001400A03F00640050083CE00000013B
:106774004000000070081A940800A001000057317E
:106784006013050083CC000000940000000010009A
:106794000400A00400210012003C2000000040007E
:1067A4000000000202940050A0006040003C202041
:1067B400010003C2000001040000069D9E000000C9
:1067C400A07BE002F100083DC0000000C000000012
:1067D40000001A9408000800C00053E000004000C4
:1067E40083DC00002008000814F510000000000FEE
:1067F40004010200403C00000000C0000000000250
:10680400029400000000E00050400000000103C0BA
:106814000F0F0008100215A79A4000402E3A0000FE
:106824000000283CC0000200000000000000183CEA
:1068340040000000000000000206500083DE00005B
:106844000000000303B080000000AD0B002C4200E8
:10685400003C20000000000000000002003C20007A
:1068640000000000000002E8200003C20000002035
:1068740014835C1180000040F216266500000000BD
:1068840000800A00000000000008183C4001E000FD
:106894000800A379E7C0200083D4081E0000000389
:1068A40080A00B000000F00B5668F000000000F020
:1068B4000580000000000000003C200000000000F3
:1068C400A080C240000003C00F1050000000000070
:1068D400000000000072206404000000008000003A
:1068E400000000000000183C6000040000000001EB
:1068F400E7910020A940080000000000000000000B
:1069040000000507A46400000000007005000000FA
:1069140000000000003C0000080000000000002807
:1069240000001680BF00000000280DE500000000F4
:1069340001F2A066F10000000078100000000000E1
:106944000000083C60380000080AA76A06040080BA
:1069540083CC00010000000406F08B0000000076E8
:106964006425020000000008F0000000000000029E
:10697400503C00080000010AA00247C0000003C008
:10698400000F140030B1CDB3800000C2D33660389C
:106994000000000000001090000000008000083C8F
:1069A40060000000104F03000040020083CE078007
:1069B40004000030C0808B000000DB02A400020051
:1069C40000000000E004000000000002503C200031
:1069D4000000000F00800328032003C20000000011
:1069E40000C3C6A0000000000A7300000000283C99
:1069F400E000000000000000020000426AD0000035
:106A040000005175E0000000006FA00B0000003C86
:106A14003E00000000800F0B40000000003C00001E
:106A2400000000000000050020005B70000000056D
:106A3400F0F1C00000010014B01E000000C3C4E562
:106A440000001400053F80000000283D60000001A4
:106A540040000000000000416B80A0814407A3E2D5
:106A640066600540ABDD8B9A0014003C000080009A
:106A74000400050000000000003C0000000040008D
:106A84000000000020024A70A000400150F843C0FA
:106A9400010016818900000400C3C4A981000040DC
:106AA4000037C0000000083DE070000880000000CE
:106AB4000008083D4050A0008423D1E56000000098
:106AC400202FAB1CA000003C010108000000800F37
:106AD400C0000000003C00080004C00000000000EA
:106AE400003C205000008802607420000000001464
:106AF400B710000000C3C4A818000040C230000052
:106B04000000083DC001E800000000000200083D4C
:106B14004038A408008767F0038000008135E81D31
:106B24004000003C010100000000C10B0000000017
:106B3400203C00000000000000000400003C20385D
:106B4400A200000347F4040000800024D9182000A8
:106B540000C3C5E000000000507336680000083D23
:106B6400C0000000000000000000409EC1180000AA
:106B74000020F700E04000000A06150E0020003C4B
:106B84000000000000000A0354000000203C0070D4
:106B94000000000000000000006F69000000000019
:106BA400F08022400020051CC090000000C3C5A056
:106BB40000000000000000040000483CC000E000A9
:106BC400000000000000083C60800000000051ACA0
:106BD40046C000110016B00F0080003C0000000009
:106BE4000000000000280000003C2090000000008D
:106BF40000000000003C00100000000AF074424055
:106C040030800081C00A014000C3C5A718000000FD
:106C14000000200400000A9400108000000000001E
:106C24000000083C60000140000A53F600400000E8
:106C34000094C7180000003C0100000000000000A0
:106C44000428000001680F09E000000000000000B3
:106C5400003C00000000000550A9C3C00000001E55
:106C6400F080000000AA85E181000C000000366974
:106C74000004083CE0000008000000000000029549
:106C84007D000000000AF32560000000007C900AEB
:106C94000000002A81000800000000001400000029
:106CA400003C2000900000000000000001543B0064
:106CB400000000005074000000000034E0180000E0
:106CC40000007200901103010100000000000000A8
:106CD40000020000000000000800000000020000A4
:106CE400000000000000000004000020000000007C
:106CF40000008000280000000000000000000001E7
:106D0400000000000000040000000001000000007A
:106D1400000000000000000000100000000000005F
:106D2400000040000000000000000000000000001F
:106D3400000000000000000000000000000000004F
:106D44000000040008000000000000000000000033
:106D5400000000000000000000000000000000002F
:106D640000000000000000004000000000000000DF
:106D7400028000000000000000000000000000008D
:106D840000000000000000000000000000000000FF
:106D940000000000000000000000000002000000ED
:106DA40004000000000000000000000000000000DB
:106DB40000000000000000000000000000000000CF
:106DC40000000000000000000000020000000000BD
:106DD40000000000000000000000000000000000AF
:106DE400000000000000000000000000000000009F
:106DF400000000000000000000000000000000008F
:106E0400000000000000000000000000000000007E
:106E1400000000000000000000000000000000006E
:106E2400000000000000000000000000000000005E
:106E3400000000000000000000000000000000004E
:106E4400000000000000000000000000000000003E
:106E5400000000000001000000000000000000002D
:106E6400000000000000000000000000000000001E
:106E7400000000000000000000000000000000000E
:106E840000000000000000000000000000000000FE
:106E940000000000000000000000000000000000EE
:106EA40000000000000000000000000000000000DE
:106EB4000200040000000000000000000000300098
:106EC40000000000000000000000000000000000BE
:106ED40000000000000000000000000000000300AB
:106EE400028004000000000000000000F000000028
:106EF400400000000000000000004000000000000E
:106F0400000000000000000000000000000000007D
:106F14000000000000000000000000003800000035
:106F2400000000000000000000000000000000005D
:106F34000000000000000000000000000000080045
:106F4400000000000000000000004000800000007D
:106F5400000000000000000000000000000000002D
:106F6400000000000000000000020000000000001B
:106F740000000000000000200000000000000000ED
:106F840000000000000000000000000000000000FD
:106F940000000000000000000000040000000000E9
:106FA4000000000010000000400030C0000000009D
:106FB40000000000000000000000000000000000CD
:106FC40000000000000000000000000000000000BD
:106FD400003C02000000001030C00000000000006F
:106FE400000000000000000000000000000000009D
:106FF4000000000000000000000000000000203C31
:1070040016018000000030C00000000000000000F5
:10701400000000000000000000000000000000006C
:107024000000000000000000000000000029409063
:107034000000001030C0000000000000000000004C
:10704400000000000000000000000000000000003C
:107054000000000000000000000000168010000086
:10706400000030C00000000000000000000000002C
:10707400000000000000000000000000000000000C
:107084000000000000000000003C000000000010B0
:1070940030C00000000000000000000000000000FC
:1070A40000000000000000010000000000000000DB
:1070B400000000000000003C16000000000030C08A
:1070C40000000000000000000000000000000000BC
:1070D40000000000000000000000000000000000AC
:1070E40000000000003C00000000001030C0000060
:1070F400000000000000000000000000000000008C
:10710400000000000000000000000000000000007B
:107114000000003C16000000000030C00000000029
:10712400000000000000000000000000000000005B
:10713400000000000000000000000000000000004B
:10714400000000000A00001030C000000000000031
:10715400000000000000000000000000000000002B
:10716400000000000000000000000000000000001B
:1071740000059B00000030C000000000000000007B
:1071840000000000000000000000000000000000FB
:10719400000000000000000000000000201400F0C7
:1071A4000000001030C000000000000000000000DB
:1071B40000000000000000000000000000000000CB
:1071C400000000000000000000000028061000007D
:1071D400000030C0000000000000000000000000BB
:1071E400000000000000000000000000000000009B
:1071F4000000000000000000000000050000001076
:1072040030C000000000000000000000000000008A
:10721400000000000000000000000000000000006A
:10722400000000000000000000080E00000030C054
:10723400000000000000000000000000000000004A
:10724400000000000000000000000000000000003A
:1072540000000000000000000000001030C000002A
:10726400000000000000000000000000000000001A
:10727400000000000000000000000000000000000A
:107284000000000000000000000030C0000000000A
:1072940000000000000000000000000000000000EA
:1072A400000000000000000000080AA040024000A6
:1072B400000000000000001030C0000000000000CA
:1072C40000000000000000000000100000000000AA
:1072D40000000000000000002AA168004003000034
:1072E40000058000000030C0000000000000000025
:1072F400000000000000000000000000000000008A
:107304003C6D000000000F00400000000000000081
:107314000A00001030C0000000000000000000005F
:1073240000000000000000000000000000023B78A4
:107334000000000030F168060000000000000100B9
:10734400000030C000000000000000000020000029
:107354000000000000000000000000000000000029
:1073640000080F000002400020000FD000000010B1
:1073740030C0000000000000000000000000000019
:1073840000000000000000000000000000000000F9
:1073940030F16800400000041EC00000000030C04E
:1073A40000000000000000000000000000000000D9
:1073B4000000000000000040006B100000080F00F7
:1073C40000000000000000050000001030C00000B4
:1073D40000000000000000000000000000000000A9
:1073E40000000000020043788000000030F16800D3
:1073F40000040000000D9A00000030C000000000EE
:107404000000000000000000000000000000000078
:10741400000000023800500000000F00404200004D
:10742400000000000000801030C0000000000000D8
:107434000000000000000000000000000000000048
:107444000102397881A0000030F12A664000000072
:1074540000000001400030C00000000000000000F7
:107464000000000000000000C00000000000000355
:10747400FC2B500000000F00404200000000000000
:107484000000001030C000000000000000000000F8
:107494000000000000000000000000000002BD48E1
:1074A400D800002030F12A604000000000000010E5
:1074B400000030C000000000000000000000800058
:1074C400000000000000000000000000000000A018
:1074D40000100F000000000100004FE00000001049
:1074E40030C00000000000000000000000000000A8
:1074F40000000000000000000000000001B00010C7
:1075040030F13800000520015EC00000000030C0EA
:107514000000000000000000000000000000000067
:1075240008000000000000000000000000080F0335
:1075340000000000000000000000001030C0000047
:107544000000000000000000000000000000100027
:10755400000000000000000001A0000030FFA800AF
:107564000000000000000000000030C00000000027
:107574000000000000000001683E50800080000010
:1075840000000410001C10000000000079424000BC
:10759400002D6DE30A00001030C000000000000060
:1075A4000000000004097DFBF18000800000000061
:1075B4000500046CF00000000053B4060000001243
:1075C4009CD00000000030C0000000000000024019
:1075D40000000000000000000000000000000000A7
:1075E40021CA01B0000000F0A4000000003E8300A6
:1075F4000900001030C00000000000053E0000003B
:107604000000000000000000000000000610016EF1
:1076140000A00000055121400000003E8FA70A0091
:10762400000030C000000000000000004000040220
:10763400380E00000000000000000040001FD800C9
:1076440002000550400280000000000018000010F5
:1076540030C000000000000000006000010935E1B6
:1076640018000000000000000000146D500000002D
:10767400055520000000000000050E00000030C089
:10768400000000000000000000000000017F000175
:10769400C800000000000000000011D000080F0026
:1076A4006D440020000282051040001030C000002C
:1076B40000000000000000000000065D000004005F
:1076C400000000000000000080F0000000F17E06D1
:1076D4008840000296C50C80000030C00000000005
:1076E4000000000000000000000000000000000096
:1076F40000000002941C00A20000069D40400020EF
:1077040001003E850E00001030C0000000000000A3
:10771400000000000000000018A0000000000000AD
:1077240001116C780004000816993B6000100000F9
:107734007DD00100000030C0000000000000000007
:107744000002000000000000000000000000002013
:1077540000FF00000000069740040400001680901B
:107764000000001030C00000000000000000000114
:107774000000000000E00000000000000242005D84
:1077840000A0000816996002800014148E90000076
:10779400000030C0000000000000000000000000F5
:1077A40003F900E00140000000000401401D10B096
:1077B4000008069340400000003FA6E19F0000102F
:1077C40030C000000000000000006800000007FA5C
:1077D40000000100000000000003E87D80000000BC
:1077E400169163660000003FED890C00000030C074
:1077F400000000000000000C000000000000000079
:1078040000000000000000000000000000200661ED
:107814000366C000400000800000001030C000007B
:1078240000000000002000000000000050000040A4
:1078340000000000000000005000000016606142DB
:10784400800000014FB00A0C00000000000000009E
:107854000000000000010000000000008080000023
:1078640000000001694C010140C00FA0C0000000ED
:10787400413FFCD0080000000000000000000000B0
:107884000000000000000000000000C00000000034
:10789400000293CB11E000C00FA1E8000003609F39
:1078A400D6A5000000000000000000000000000059
:1078B40000000000000000000000000000000000C4
:1078C4000028000000000C396C001080250057AB24
:1078D4000804000000000000000000000000000098
:1078E4000000000000000000000000000500057C0E
:1078F4000180001028BDF406080000801CDB800015
:107904000000000000000000000000000000000370
:107914000C7C00F000000000000000002830000093
:1079240000010E33B74000000032C3B000408000B5
:1079340000000000000000000000000000098E7B31
:107944000090880000000100000029EA0080200067
:10795400283DA74600803030CDF188A30000000008
:10796400000000000000000000000000000000C053
:107974000000000000700402BC0A000000000000C7
:1079840000000000000001F580000000000000007D
:1079940000000000000000000000000000100000D3
:1079A40000000000021A815A00000000000000607C
:1079B400001000014FC39A00000000000000000006
:1079C40000000000000000436B7908000000000084
:1079D400000000403C2A308000000000E802D00093
:1079E40000000FE180000000000000000000000023
:1079F400000000000008947A50000000000000001D
:107A04000318AD4E80F000000053A162A8000000EE
:107A140055AF0E0000000000000000000000000050
:107A2400010000000000B10000000000000200039B
:107A3400E80000A0000000000023862000000000F1
:107A440010000000000000000000000000000280A0
:107A54000000000080A00000000000010003E968AD
:107A640018A00000000001E00040000000038C00AA
:107A740000000000000000000000000000000011F1
:107A84007C08900201000000000008203D4800002E
:107A9400004105B03442400100029ED300000400BE
:107AA400000000000000000000000000000ABD40CB
:107AB4008180014000000000084A3BDA00000144D4
:107AC400ADB1EF404005000126980000140000000D
:107AD40000000000000000000000000000000000A2
:107AE400080000000030000291CB00D000000C37E9
:107AF400EFC2C600000000000D00000000000000FE
:107B04000000000000000000000000001980044094
:107B1400000000000041696800B000000631B208AE
:107B240020000000000001800000000000000000B0
:107B340000000B4040000040003F00000000000037
:107B44000000000006E9B8D000000080A02000007A
:107B54000003FE9B10000000000000000000000570
:107B640077802800000015CC780000C000000000D9
:107B7400080001FFF9D000148003B542000002039D
:107B840085FD0E000C000000000000000000B7C2DC
:107B9400000800000000B98020000000000000037D
:107BA400BEEC000020800AF03DC700800000000FFA
:107BB4000002000000000000000080013B142010BF
:107BC40000000000F9E1800000000000000179E9F4
:107BD4007980008005F50607430000000008004096
:107BE4000000000000000000000A0AC0400000007D
:107BF400000031F000000000000200000039F880AD
:107C040000000580F44003000000000300000000B1
:107C14000000000000008205500028080000000059
:107C240080E0200000000005000029DD9000200411
:107C340005A5E54001800000000D9E020000000043
:107C44000000000000050ACE00000003C000D0E0E0
:107C54000000000000000052901DB09000000807D2
:107C6400600280500030E7B0000C0000000000000B
:107C74000000060A502E00080803C0C081900000CE
:107C8400000000000110014DF8100000000D344008
:107C940000280018EE80000800000000000000002A
:107CA40000AF06C028000001603B30000000000067
:107CB400000000000358B0020000000000000000B3
:107CC400050FC0B90900000000000000000002A078
:107CD40052940000010169E950000800000000000E
:107CE400000202DF81840000000001E00000108F28
:107CF40046978800000000000000000000F3081C04
:107D04000000000020CE000000000000010000027E
:107D1400D5EF00BA0000000001C28000001780F017
:107D24008000000000000000000040F350266000C6
:107D3400000002EE18000000000002800803D6FED6
:107D4400180CC000000000000300100757D7000003
:107D5400000000000000000000811E94000050415B
:107D64006C190000004000000200044120100100D2
:107D7400004040003D4740400016C3FF0800040097
:107D840000000000000000A1DE402800510B6CCA76
:107D940000C4014000000000011921C81080014402
:107DA400001720024020102957D7010014000000BA
:107DB400000000000000000000700003974D7000F8
:107DC4000000000000000202836A100008000000A6
:107DD400BC038500040F17EB8F4000000000000077
:107DE40000000000000000000000966D90000000FC
:107DF40000000000000340EB80A0100000553C0090
:107E04000000000E3D9D0020000000000000000066
:107E14000000F68020000241403F71D0088000003D
:107E2400000000400A7C790000000FA03E4340009F
:107E340000210DD90004080000000000000000101B
:107E4400728004000011685A50D0108000000000B5
:107E54000000027E50C000C00F55046040000020A6
:107E64007CF8008008000000000000000050074477
:107E740000000042BC0A700400000000000000037F
:107E84000EEB010400000CBD2064000000000000A3
:107E940000004000000000000000020A12E0600040
:107EA4000000155C000A000000000000000A2EDC3F
:107EB400018200000C3BFD460300000000058E001B
:107EC400000000000000000000A002C4000008013F
:107ED4007C0E50080000000000000001683B1900FF
:107EE40000000F008000005000028300100000001A
:107EF400000000000000030A16A00000000014CBDC
:107F040001C0000000000000010290EBD0C000009E
:107F14000F070003010000028CA50C000000000004
:107F24000000000000A0024000000000000000C0AB
:107F340000000000006000016C2B00E00000000065
:107F4400A5C000000000000B0000000000000000BD
:107F54000000030A17800000000000000000000079
:107F64000000000001029559119140180057300695
:107F740080000000000180000000000000000000FC
:107F840000A006C0000008030E6800000000000006
:107F940000000000140FD800000000F06822400028
:107FA400004282DD00000800000000000000030A17
:107FB40012806000000B1DFE500000000000000055
:107FC400000029C17180000400D5FCE6C000408196
:107FD4004C080001480000000000000000A00674E6
:107FE40020000800142001E000000000000000430D
:107FF400C00058040000000938020000440F03D1F7
:10800400001C0000000000000000030A13860400A6
:10801400000015E801E00000000000400003C0C0BB
:10802400900A0000080D6002C000100F5EA59800C1
:10803400000000000000000000A002C00000420395
:10804400FC2800900100000000000003C40CF8B1FB
:1080540000400F008143C70000140290080144004F
:10806400000000000000030A13800000400814FE12
:108074000000010000000000011BD17878A001403D
:108084000F030002C00000168D8000009400000061
:108094000000000040A0027420000000000010F066
:1080A400000000000000000081FC0000000300F05C
:1080B40002C00000040F17D0000000000000000000
:1080C4000000030A1280000000000000198008402C
:1080D40000000000000002F80000002000F102008F
:1080E4000004040F57E580000000000000000000B9
:1080F400000000000000004002F801D10000000070
:1081040000100003FC3E0890000000054000002021
:10811400001001D9890000000000000000000000E8
:10812400000000003002917F79D0000000000000C0
:108134000003E8DF38C000001008204000501100A0
:108144001FE38C000C000000000000000000000091
:108154000000000000000000000000000000000318
:10816400FF48F0B00428069F00E000000002EDF094
:10817400900000000000000000000000000000501B
:108184000000000001E00000000000000001FDDD2F
:1081940080000800169160C00820000167C1080132
:1081A4004000000000000000000000000004020085
:1081B400003C09000000000000000000015D010017
:1081C4000020469F01400800000000099000800044
:1081D4000000000000000000000000720100047BA9
:1081E40079E00000000000000000066B19C00008E0
:1081F400169129C01000000000011E01400000007B
:10820400000000000105080000000000003F3000ED
:108214000000000000000003FF6B7000000846939C
:10822400400700002017C0838000200000000000E9
:108234000000020556800000000014F919C0000077
:10824400000000220003F97B0180000816916002FF
:10825400000000A95E9B0000000000000000000078
:10826400000000002000002316EB70000000000056
:1082740001000200001F70A0000006910002C0006F
:10828400000FC29080800000000000000000000089
:1082940000000400021B004FB00000000000028038
:1082A4000100117899B20000169160004000D0AF2F
:1082B400D695000000000000000000000000001C33
:1082C400200000100750010000000000000000031F
:1082D400E800000080000EDF6C068600001FDCB0A2
:1082E4000000000000000000000000000020040066
:1082F400000006EC00800000000000020003E968B2
:108304003000000017B97062C000001E9E8180001A
:108314000000000000000000000000000000100247
:10832400E80CF0005440000002000001400850F046
:108334000020869340268000201542008800040017
:108344000000000000000000000000005120695EF1
:10835400B8C0014000000104000281E08010000068
:10836400169171C28000011554811F001400000091
:10837400000000000105080000000001542DF80071
:108384000000000000000800025A000000000F0175
:10839400804200000030C6D0180000000000000039
:1083A40000001205528000000002945EF8000000F4
:1083B40000000000000006CF01A000001F012B6296
:1083C400F00400A2DFC01D1C00200142E00B0000ED
:1083D40000000000000002217C303800140000007E
:1083E40000000003F40F7900000043F0A0074020D0
:1083F4008029A7C108000000028C100000000000C2
:108404000000000000017DDA700008000000000098
:108414000103697EB1C000D423D17842401300A97E
:1084240077E9801800000000000000000000000050
:1084340000000000000008F0000000000000000040
:10844400003FF09000000FC020000000001680AD37
:108454009000000000000000000000000000000088
:10846400000000003810000000000002000014DDCD
:10847400800000040585F942000000A940010C10A9
:1084840000000000000000000000000000000001E7
:108494007C3C00901000000000000000F82CB0D0DC
:1084A40000000C29E167000000004F90000040002C
:1084B400000000000000000000000000000014DEC6
:1084C4000180C80000000070074AF0FBB2E0000819
:1084D400081BBDC30000000006E00000800000008F
:1084E4000F0000000000000C00000000143F110009
:1084F4000000000000000001683B7800000004A5B3
:108504006020000000300200180000000000080095
:1085140000000000002000000002BD5901C000005E
:10852400000000200102917FB9E100002AD7E44055
:10853400000011B01C000F00000000000000180033
:108544000000000000400001542B50820000000095
:10855400000400016CEE7000000000000002000046
:108564000020C2E000A0C0000000000000000000E5
:1085740000000000000295E9101200000000000253
:10858400000294DC9980000000000060402010008C
:108594000795004C400000000000000000000000AF
:1085A4003C002020980C5000000000000000000057
:1085B400003F000000000C3D70000B1000061E8000
:1085C400004800000000000000000000000004005B
:1085D4003108F57D0000000000000000001014DDEB
:1085E40000001400063BA4039000000B84D0080094
:1085F4000000000000000000000000000000100067
:10860400A80900F14040000000000203C00000007F
:1086140000400F00802600010003C005080004008C
:108624000000000000400000000000804101E8F864
:1086340078100140000000000003C1600001014007
:108644000F0580E241050083CC0581001400000081
:108654000000000000F0000000000002BC2F00D069
:10866400000000000280000000000000000000F78D
:10867400FC6200000003C200000140000000000092
:10868400000006F050000000000015EF1810000074
:1086940000000100000000000008000000E3B7E350
:1086A400C0000083DE010000C000007200801100E1
:1086B40062002F8200000103D7D728080000F7D3F7
:1086C4000C240200F3F708000002FFFF0000010180
:1086D400BFBF44042020FBFB04142020EBEF100058
:1086E4000420FDFD02004004FFFF00000040EFEF06
:1086F40010200000F7DF28088584F7DF200400013C
:10870400DBEB1C188000E7F700080080F7FF080087
:108714000202FFF30C0C0200F3F30C080002F7F75B
:1087240008080000F7F708000000FFF71008000031
:10873400C7EF20000400EFCF31110004EDCE360462
:108744000000DBF90A0C0000FFF500020000FFFF47
:1087540000000404FBFB04000000FFFF0000000015
:10876400EFFF10100000CBEF24242000FFFB0000DB
:108774002020FFFF00082020E5F613190100FDED7D
:1087840002220001FDD52A0A0000DFDD22000000DC
:10879400FBDF04240000FFFB00000000FFFF0404D3
:1087A4000000FFEB10100000CFDF22020101FFFDEB
:1087B40000000000FFFF08080000FEE6111242005E
:1087C400EFFD02000042F7F50E000202F9FB00047F
:1087D4000000FFFF08002120F7F700082021F3FB29
:1087E4000C141020EFE718081414F7F50A0A505077
:1087F400F7F708081010F7F708101010EDE7120843
:108804009511F7FD02001094FFFD06049090F1F31A
:1088140008001010FFFF00000210BFBF4404020252
:10882400FBFB14100000EFEF00100000FDFD020040
:108834000000FFFF00000000EFEF10100404F7FF3A
:1088440008080000F7FF00000000EFFB1C1E0000FA
:10885400E3E50A0A0000F5F50A0A0400F5F10E043E
:108864000004F9F300080000F7FF00000000FFFF18
:1088740000000000FFEF10102000FFEF0000202098
:10888400E7ED130B2020FDEC12160101F9E90E0AA5
:108894000000FDF502020000FDFD02000000FBFBEC
:1088A40004000000FFFF00100000EFEF10100100B3
:1088B400EFFB04040001FBFF00000000FFFF0A00BF
:1088C4000000F5F4130B0000EDED12004242FFF539
:1088D4000A080002FDFD02023020FDFD06003030D2
:1088E400FBFB00041111FFFB14041410EBEF100048
:1088F4005014DFDF22021050FFFD00001010FFFFB4
:108904000A081110FCF413121011EDED12029494E4
:10891400F5F50A021090F9F906021010FFFD08009F
:108924001210F7F7080C1212E3F3181C1010E7E703
:1089340008080010FFF50A020000F7FF0000040019
:10894400FDFF02020004FDED12120000FDED020223
:108954000000F5FD060A0000F1F10A0E0000FDFF1B
:1089640000000000FFFF04040404EBEB10140000FB
:10897400EFFF00000000FDFD02000000FFFF00000B
:108984000000FFEF10100000EFF708082020FFFFA1
:1089940000022120FDFD0E160001E5E11A10000081
:1089A400E7FD02080000FDF906060000FDF90200DB
:1089B4000000FFFF0000010100008200800103FFAE
:1089C400FF10000000EFEF10000000FFFF0208009E
:1089D40000E5E51B030000FDFE10005202EFEB1C56
:1089E4001C3052E3F700023030FFFD02021010F990
:1089F400F904121110FFEF10100415EFEF001040EE
:108A040040FBFB04000000FFFF00000000FDFD0A26
:108A1400020101F7F401030000FFEF10108400E7E6
:108A2400EF08180004F7FF00020000FDFD02061223
:108A340002FBF914001210EFEB14141012FFEF00F4
:108A4400001010DFDF22021010FFFD00000414F5F7
:108A5400FD0A0A0000F6FC01020000EFEF1010000E
:108A640000F7E708100000FDFB06040000FDFD020E
:108A74000A0000E5F71C000400E3EB10180004EF03
:108A8400FF00000000FFFD02020000FFFF020000E3
:108A940000FDFD02020000FFFD10020000EBEF10DC
:108AA400142020F7E30C120121F3F10E0A0000F563
:108AB400FD02100000FFEF14140000EBEB100001A6
:108AC40000FFFF00000001FDFD02000000FFFF00A9
:108AD400000000EFFF10101000F7E708001210FF6D
:108AE400FD02023012FDFD040A7272F3E310180055
:108AF40010EFEF10000000EFFB04060400FBFD0282
:108B0400024105FDFD00120040EFEF10100000FFD0
:108B1400EF00000100FFFD0A020001E7E511090072
:108B240000FFFE00000000FBEF1C140404E3E71048
:108B3400180200EFEF10120002E9E916120000ED2E
:108B4400EF10000202FFFF00041000FBFB00041002
:108B540010FFFF02001010FDFD0A081010FFF601BF
:108B6400010010FFFF00100000E7EF18180000EFED
:108B7400E710140000EFEB16100000E9E9161400EA
:108B840000EBEB04100000FFFF00000000DFDF2219
:108B9400020000FFFD02020000FDF50A080000F6D5
:108BA400FE01000000FFFF10000000E7E71810219D
:108BB40020EBEF14140021E9EF12120000E5E51C8C
:108BC400140000FBEB00000101FFFF00000000FFA8
:108BD400FD02020000FFFD02061000FBFD04001070
:108BE40010FFFB04041212EBFB141C2030E3E31C03
:108BF400144220E3E31C180042EDE512120000EDDC
:108C0400EF14140000EFFB00004140FFFF000000E0
:108C140001FDFD02000000FFFF00000101FFFF183D
:108C2400000000E7E712180000EDFD02000000FF5D
:108C3400FF04000000F3F3081C0202EFEF10100021
:108C440000EFEB14140000EFEF10120200EDED1230
:108C5400120002EFEF10000000FFFF02001000FD01
:108C6400FD0A081010E7E711011010FFFE000000D4
:108C740010FFFF040C0000E7F318000000FFEF10E2
:108C8400000000F9EB06120000EDFD00000000FFFB
:108C9400FF04000000FBFB00000000FFFD020200D7
:108CA40000FFF508080000F7FE01050000FBFF04C3
:108CB400000000FFFB0C142000F3E3140421210046
:108CC40000110162003F8200000103000000000067
:108CD4000000001B1B0000000000001F1B00000020
:108CE400000000041F00000000000000000000005D
:108CF4000000001B000000000000001B1B0000001F
:108D04000000001F1B0000000000001F1F000000E7
:108D140000000000000000000000001B1B00000019
:108D24000000001B1B0000000000001F1F000000CB
:108D34000000001F1F000000000000001B000000D6
:108D44000000001B1B000000000000001B000000CE
:108D540000000004040000000000001F1F000000C9
:108D6400000000001B0000000000001B1B000000AE
:108D7400000000E4FB000000000000E4E400000048
:108D84000000001FFF000000000000001B000000A6
:108D9400000000F919000000000000E4F9000000E0
:108DA400000000E4E4000000000000F7F700000009
:108DB4000000000013000000000000F9F9000000AA
:108DC400000000E4F9000000000000E4E4000000FA
:108DD400000000F7F700000000000000F3000000AE
:108DE400000000F9E900000000000014FD0000008C
:108DF4000000001E1C000000000000F7FF0000003F
:108E040000000000E1000000000000E9E9000000AB
:108E14000000001CFD0000000000001E1A000000FD
:108E2400000000EFFF00000000000000E10000006F
:108E3400000000DDC90000000000001EDD0000008D
:108E44000000003E3A000000000000BDBF0000002A
:108E540000000000A9000000000000DDD9000000AF
:108E6400000000A2FF000000000000A6A200000015
:108E7400000000BDBD00000000000000B9000000BB
:108E8400000000FFDD000000000000A6FF0000005D
:108E94000000008486000000000000BDBD0000004A
:108EA40000000000BD000000000000FFFD00000005
:108EB40000000006FF0000000000000404000000A1
:108EC4000000003D3D000000000000003D000000E7
:108ED400000000FFFF00000000000006FF0000008B
:108EE4000000000404000000000000FDFD0000007C
:108EF40000000000FD000000000000FBFB0000007B
:108F040000000000FB00000000000024000000003E
:108F1400000000FDFD00000000000000F90000005A
:108F2400000000FBFB000000000000FBFB00000051
:108F3400000000FFFB000000000000FFFF00000035
:108F440000000000FB000000000000FB2200000005
:108F5400000000FBFB000000000000DFFB0000003D
:108F6400000000FFFF0000000000000022000000DD
:108F74000000002202000000000000FBFB000000D3
:108F8400000000DFDB00000000000026FF000000FE
:108F940000000000220000000000000000000000AB
:108FA40000000000000000000000000000000000BD
:108FB40000000000000000000000000000000000AD
:108FC400000000000000000000000000000000009D
:108FD400000000000000000000000000000000008D
:108FE400000000000000000000000000000000007D
:108FF400000000000000000000000000000000006D
:10900400000000000000000000000000000000005C
:10901400000000000000000000000000000000004C
:10902400000000000000000000000000000000003C
:10903400000000000000000000000000000000002C
:10904400000000000000000000000000000000001C
:10905400000000000000000000000000000000000C
:1090640000000000000000000000000000000000FC
:1090740000000000000000000000000000000000EC
:1090840000000000000000000000000000000000DC
:1090940000000000000000000000000000000000CC
:1090A40000000000000000000000000000000000BC
:1090B40000000000000000000000000000000000AC
:1090C400000000000000000000000000008200809A
:1090D40001032C2C0000000000001F3E00000000D3
:1090E40000009F1F000000000000CCDE0000000014
:1090F400000000480000000000003E2C00000000BA
:1091040000001F3F0000000000009F9F00000000BF
:109114000000DEDE00000000000000480000000047
:1091240000003F3E0000000000009F3F00000000E0
:1091340000009F9F000000000000DEDE0000000031
:109144000000005A00000000000037360000000054
:109154000000813700000000000089810000000049
:1091640000005A5A000000000000005200000000F5
:109174000000F636000000000000C1F60000000008
:109184000000A981000000000000FAFA00000000BD
:1091940000000052000000000000F4740000000011
:1091A4000000C1F4000000000000A9E90000000074
:1091B4000000F2FA0000000000000072000000004D
:1091C4000000F474000000000000E5F4000000005A
:1091D4000000EDED000000000000F2FE00000000C1
:1091E4000000007200000000000074740000000021
:1091F4000000A774000000000000CF8F00000000F2
:109204000000767E000000000000007000000000F6
:10921400000074740000000000009F74000000004F
:1092240000009F9F00000000000074760000000012
:1092340000000074000000000000746400000000DE
:1092440000009B740000000000009B9B00000000D5
:1092540000007676000000000000007400000000AA
:109264000000606000000000000099700000000031
:1092740000008999000000000000767600000000DC
:1092840000000076000000000000606000000000A4
:1092940000008960000000000000898900000000CF
:1092A4000000767600000000000000760000000058
:1092B40000006464000000000000896C00000000ED
:1092C40000008189000000000000767600000000A4
:1092D4000000007600000000000076760000000028
:1092E4000000897E00000000000081890000000069
:1092F4000000767600000000000000760000000008
:1093040000007676000000000000A97E0000000046
:109314000000C18900000000000076760000000013
:1093240000000076000000000000777600000000D6
:109334000000FF7F000000000000F7FF00000000B5
:1093440000007777000000000000007600000000B5
:1093540000007760000000000000DF7F00000000D4
:109364000000B7FF00000000000077770000000055
:109374000000006000000000000061200000000008
:109384000000DF7F000000000000B79F0000000025
:1093940000006177000000000000004000000000B1
:1093A40000000000000000000000000000000000B9
:1093B40000000000000000000000000000000000A9
:1093C4000000000000000000000000000000000099
:1093D4000000000000000000000000000000000089
:1093E4000000000000000000000000000000000079
:1093F4000000000000000000000000000000000069
:109404000000000000000000000000000000000058
:109414000000000000000000000000000000000048
:109424000000000000000000000000000000000038
:109434000000000000000000000000000000000028
:109444000000000000000000000000000000000018
:109454000000000000000000000000000000000008
:1094640000000000000000000000000000000000F8
:1094740000000000000000000000000000000000E8
:1094840000000000000000000000000000000000D8
:1094940000000000000000000000000000000000C8
:1094A40000000000000000000000000000000000B8
:1094B40000000000000000000000000000000000A8
:1094C4000000000000000000000000000000000098
:1094D40000000000110262002F820000010300005E
:1094E4000020000000000022000000000022000014
:1094F40000000002000000000022000000000066DE
:10950400000000000066000000000066000000008B
:10951400006200000000004400000000004400005D
:109524000000003700000000004400000000006458
:10953400000000000076000000000063000000004E
:109544000046000000000066000000000037000034
:1095540000000046000000000062000000000066F9
:10956400000000000046000000000026000000008B
:1095740000620000000000260000000000640000FB
:1095840000000066000000000066000000000040CB
:10959400000000000044000000000044000000003F
:1095A400000400000000006600000000000000004D
:1095B40000000066000000000020000000000046DB
:1095C4000000000000200000000000420000000035
:1095D40000260000000000000000000000620000FF
:1095E40000000064000000000046000000000024A9
:1095F40000000000004600000000002200000000FF
:1096040000200000000000460000000000200000D0
:1096140000000002000000000044000000000044BC
:109624000000000000660000000000400000000090
:1096340000260000000000200000000000020000DE
:1096440000000020000000000002000000000022D2
:109654000000000000440000000000620000000060
:10966400000400000000002200000000004400008C
:10967400000000440000000000330000000000442B
:109684000000000000600000000000160000000060
:1096940000610000000000060000000000660000F9
:1096A400000000110000000000440000000000223F
:1096B400000000000044000000000044000000001E
:1096C400002200000000004000000000002600000E
:1096D40000000060000000000046000000000004DC
:1096E4000000000000000000000000440000000032
:1096F40000440000000000000000000000660000BC
:1097040000000000000000000066000000000020CF
:1097140000000000006600000000002200000000BD
:1097240000560000000000230000000000000000BC
:109734000000002200000000006400000000004659
:1097440000000000002000000000004600000000AF
:10975400002200000000002000000000006600005D
:109764000000002200000000000200000000004091
:10977400000000000044000000000026000000007B
:109784000040000000000004000000000020000071
:1097940000000002000000000020000000000002A1
:1097A400000000000022000000000044000000004F
:1097B4000022000000000000000000000022000061
:1097C4000000000000000000000000000000003362
:1097D4000000000000000000000000200000000065
:1097E400820080010300000032000000000023001A
:1097F4000000000002000000000022000000000041
:109804001100000000000000000000002200000021
:109814000000000000000000000000000000220022
:109824000000000000000000000022000000000012
:109834002000000000000200000000000000000002
:109844000000000000000000000000000000000014
:1098540000000000000000000000220000000000E2
:1098640000000000000022000000000020000000B2
:10987400000022000000000022000000000056004A
:1098840000000000230000000000000000000000B1
:109894002200000000002000000000000200000080
:1098A4000000200000000000020000000000220070
:1098B4000000000020000000000022000000000062
:1098C4002200000000000200000000000000000070
:1098D4000000000000000000220000000000000062
:1098E4000000000000000000000020000000000054
:1098F4000200000000002000000000000200000040
:1099040000003300000000005400000000002300A9
:109914000000000000000000000033000000000010
:1099240011000000000020000000000013000000EF
:1099340000001000000000002100000000003200C0
:1099440000000000230000000000130000000000DD
:1099540022000000000011000000000000000000D0
:1099640000003300000000001100000000000000AF
:1099740000000000220000000000000000000000C1
:10998400320000000000310000000000030000006D
:1099940000000000000000001100000000001100A1
:1099A40000000000000000000000110000000000A2
:1099B400320000000000010000000000320000003E
:1099C4000000210000000000020000000000000070
:1099D4000000000010000000000023000000000050
:1099E400000000000000330000000000310000000F
:1099F400000002000000000031000000000012001E
:109A040000000000230000000000310000000000FE
:109A1400120000000000010000000000100000001F
:109A240000001100000000000100000000003200EE
:109A340000000000010000000000330000000000EE
:109A440020000000000002000000000020000000D0
:109A54000000020000000000330000000000550078
:109A640000000000330000000000100000000000AF
:109A7400330000000000110000000000210000007D
:109A8400000013000000000011000000000031007D
:109A9400000000001200000000001100000000009F
:109AA400110000000000230000000000110000006D
:109AB400000010000000000033000000000011004E
:109AC400000000000100000000002200000000006F
:109AD400000000000000330000000000310000001E
:109AE40000001300000000110362003F8200000127
:109AF400030000000000000000000000000000005F
:109B04000000000000000000000000000000000051
:109B14000000000000000000000000000000000041
:109B24000000000000000000000000000000000031
:109B34000000000000000000000000000000000021
:109EF4000000008200800103000000000000000058
:109F0400000000000000000000000000000000004D
:109F1400000000000000000000000000000000003D
:109F2400000000000000000000000000000000002D
:109F3400000000000000000000000000000000001D
:10A2F400000000000000000000002206DE0106004D
:10A30400040000000103000001000000010000003F
:10A3140003000000010000000F0000000F00000017
:10A324000000000036A500080018024010000000DC
:10A33400060400003BA500080018024008000000C5
:10A34400060301003EA500080018024002000000B8
:10A354000601010045A500080018024004000000A1
:10A36400060201000000000000000000005400404C
:10A374000004024040000000060004000004024003
:10A38400000200000900040000002000801A0600FA
:10A39400004000001F20000000000000000000003A
:10A3A40000580040001402400200000001000400B4
:10A3B40000140240010000000000040000004000FE
:10A3C400801A0600FFBF00002122000000000000E8
:10A3D400F513000801000300820007008400070051
:10A3E4000100030002000300400003008000070096
:10A3F40084000700000001000000000000000008C5
:10A40400004000080080000800C0000800000108A7
:10A414000000020800000408000006080000080804
:10A4240000000A0800000C0800000E0800000800E4
:10A4340010001800200028003000380040004800B8
:10A4440050005800537475636B20627574746F6E9A
:10A4540020726567697374657220697320696E760A
:10A46400616C69642C20636C656172696E672E008F
:10A47400427574746F6E20697320707573686564B7
:10A4840020617420626F6F740069636534306C708E
:10A494002E630043444F4E45206E6F74206C6F77DB
:10A4A40020647572696E6720726573657400435227
:10A4B40045534554206E6F7420686967682064753D
:10A4C40072696E6720726573657400446973706C99
:10A4D400617920627573792D776169742074696D6F
:10A4E400656F7574206578706972656421004469CC
:10A4F40073706C617920696E697469616C697A65DD
:10A5040064206166746572200020726574726965E6
:10A51400732E00446973706C617920696E69746983
:10A52400616C697A6174696F6E206661696C6564D7
:10A534002E004261636B0055700053656C65637453
:10A5440000446F776E006372632E63006932632E7A
:10A554006300493243206465766963652049442079
:10A564006F7574206F6620626F756E647320256446
:10A5740020286D61783A20256429006F6E0073707D
:10A58400692E6300206973206F7574736964652094
:10A5940073797374656D20666C6173680D0A00735A
:10A5A400797374656D5F666C6173685F65726173FE
:10A5B4006528002C2000290D0A006661696C656419
:10A5C40020746F20657261736520736563746F72A4
:10A5D400200073797374656D5F666C6173685F776F
:10A5E4007269746528006661696C656420746F2003
:10A5F40077726974652061646472657373200049BD
:10A604006E76616C6964206669726D77617265202B
:10A614006465736372697074696F6E210043686561
:10A62400636B73756D6D696E67206669726D7761B2
:10A6340072652075706461746500496E76616C6939
:10A6440064206669726D77617265204352432069A4
:10A654006E2053504920666C6173682100657261F5
:10A6640073655F6F6C645F6669726D7761726500B4
:10A6740077726974655F6E65775F6669726D77611D
:10A68400726500436865636B73756D6D696E6720F1
:10A69400002062797465730D0A00436865636B7307
:10A6A400756D202D2077616E746564200020676FBE
:10A6B4007420004F757220696E7465726E616C202F
:10A6C400666C61736820636F6E74656E7473206169
:10A6D4007265206261642028636865636B73756DBD
:10A6E400206661696C656429212054686973206956
:10A6F40073207265616C6C792062616421004F750E
:10A70400722070726576696F7573206669726D77F1
:10A7140061726520757064617465206661696C6539
:10A72400642C2061626F7274696E67207570646155
:10A7340074652E004E6577206669726D7761726567
:10A7440020697320617661696C61626C6521004CDB
:10A754006F6164696E67207265636F7665727920D4
:10A764006669726D77617265004661696C65642023
:10A77400746F206C6F6164207265636F76657279A3
:10A78400206669726D776172652C20737472696BCF
:10A7940065206F6E652E2054727920616761696E41
:10A7A4002E004661696C656420746F206C6F61646F
:10A7B400207265636F76657279206669726D776160
:10A7C40072652C20737472696B652074776F2E2008
:10A7D40054727920616761696E2E004661696C6507
:10A7E4006420746F206C6F6164207265636F76659A
:10A7F4007279206669726D776172652C2073747248
:10A80400696B652074687265652E20534144205736
:10A81400415443480048415244204641554C540059
:10A8240065786974207374616E64627900205F5F77
:10A834005F5F202020202020202020202020202096
:10A84400205F5F002F5C20205F605C2020202020A0
:10A854002020202020202F275F5F605C005C205C8C
:10A864002C5C4C5C5F5C202020205F5F5F202F5CB1
:10A87400205C2F5C205C20205F5F20205F5F202015
:10A884005F5F20205F5F20205F5F00205C2F5F5CA4
:10A894005F5F205C20202F27205F20605C205C20ED
:10A8A4005C205C205C2F5C205C2F5C205C2F5C2097
:10A8B4005C2F5C205C2F5C205C002020202F5C201F
:10A8C4005C4C5C205C2F5C205C2F5C205C205C205A
:10A8D4005C5F5C205C205C205C5F2F205C5F2F2031
:10A8E4005C205C205C5F5C205C002020205C20609D
:10A8F4005C5F5F5F5F5C205C5F5C205C5F5C205C36
:10A904005F5F5F5F2F5C205C5F5F5F785F5F5F2FDF
:10A91400275C2F605F5F5F5F205C00202020205C4D
:10A924002F5F5F5F5F5F2F5C2F5F2F5C2F5F2F5C5C
:10A934002F5F5F5F2F20205C2F5F5F2F2F5F5F2FC4
:10A94400202020602F5F5F5F2F3E205C00202020AE
:10A9540020202020202020202020202020202020F3
:10A9640020202020202020202020202020202020E3
:10A9740020202020202020202F5C5F5F5F2F0020DC
:10A9840020202020202020202020202020202020C3
:10A9940020202020202020202020202020202020B3
:10A9A400202020202020202020205C2F5F5F2F00EB
:10A9B4004C617374206669726D7761726520626F91
:10A9C4006F742077617320737461626C653B2063DC
:10A9D4006C65617220737472696B657300486F6C87
:10A9E4006420646F776E205550202B204241434BE6
:10A9F40020666F72203520736563732E20746F2078
:10AA0400666F7263652D626F6F7420505246004604
:10AA140069726D776172652069732065726173650F
:10AA240064005761746368646F672063617573655C
:10AA340064206120726573657400536F6674776176
:10AA44007265206661696C757265206361757365F2
:10AA5400642061207265736574004661696C656485
:10AA640020746F207374617274206669726D7761EB
:10AA740072652C20737472696B65207468726565E5
:10AA84002E004661696C656420746F207374617272
:10AA940074206669726D776172652C2073747269B3
:10AAA4006B652074776F2E004661696C6564207451
:10AAB4006F207374617274206669726D7761726558
:10AAC4002C20737472696B65206F6E652E00426F63
:10AAD4006F74696E67206669726D77617265204074
:10AAE40020002E2E2E0D0A0D0A00466F7263652D6E
:10AAF400626F6F74696E67207265636F76657279D1
:10AB0400206D6F64652E2E2E00536F66747761720C
:10AB140065206661696C7572653B20726573657446
:10AB240074696E6721004153534552543A20002002
:10AB340020003A0041535345525400415353455267
:10AB4400544E002A2A2A20575446200053544D3389
:10AB5400320053544D3332207065726970686572E7
:10AB6400616C206C696272617279207472697070B0
:10AB7400656420616E206173736572740043524F83
:08AB8400414B204F4F4D000032
:10AB8C00FF00000000010203040102030406070891
:04AB9C0009000000AC
:04000005080001B43A
:00000001FF
